:100000000C9436000C94D3060C9400070C945E00FC
:100010000C945E000C945E000C945E000C945E00E8
:100020000C945E000C945E000C945E000C945E00D8
:100030000C945E000C945E000C945E000C945E00C8
:100040000C942D070C945E000C94D7070C94250893
:100050000C945E000C945E000C945E000C945E00A8
:100060000C945E000C945E009B00910911241FBE4D
:10007000CFEFD8E0DEBFCDBF11E0A0E0B1E0E4EF0C
:10008000F8E102C005900D92A239B107D9F713E04B
:10009000A2E9B1E001C01D92AC32B107E1F710E076
:1000A000CCE6D0E004C02297FE010E94740CC83652
:1000B000D107C9F70E94E7090C94780C0C94000052
:1000C000CF93DF93EA01EBEBF1E020E030E00CC0EE
:1000D00060FD02C040E301C041E341932F5F3F4F09
:1000E00096958795779567956115710581059105B9
:1000F00079F7AE01421B530BDE01A654BE4FEBE96C
:10010000F1E020E030E090E30BC02417350718F051
:100110008C91808301C090832F5F3F4F1197319660
:100120002C173D0790F3C556DE4F18828BE991E0FE
:10013000DF91CF91089582E991E00E94E601089550
:100140004F925F926F927F928F929F92AF92BF92E7
:10015000CF92DF92EF92FF920F931F93DF93CF9393
:10016000CDB7DEB7E2970FB6F894DEBF0FBECDBFB6
:100170005B016C014A013901502E412E6115710558
:100180008105910539F48AE093E060E071E00E9416
:10019000FD0A86C00E946000182F092F8AE093E0B4
:1001A00062E171E00E94FD0A8AE093E0B601A501D8
:1001B0002AE030E00E94C00A8AE093E06CE171E03E
:1001C0000E94FD0A8AE093E0B4014AE050E00E94F8
:1001D000CF0A8AE093E06FE171E00E94FD0A8AE0B5
:1001E00093E0612F702F0E94FD0A8AE093E06DE298
:1001F00071E00E94FD0A212F302FC9019C01BE0130
:100200006F5F7F4FA0E0B0E046E419C0903319F46F
:10021000803341F404C0913351F4813341F4FB0144
:10022000808308C0813319F4FB01408303C06AE373
:1002300071E012C011962E5F3F4F6F5F7F4FF90143
:100240009081992319F08181882301F7CE010196CD
:10025000A80FB91F1C92BC018AE093E00E94FD0A1E
:100260008AE093E069E471E00E94FD0A8AE093E08D
:10027000B3014AE050E00E94CF0A8AE093E068E5CB
:1002800071E00E94FD0A8AE093E066E671E00E9458
:10029000FD0A8AE093E0B7014AE050E00E94E00ADC
:1002A0008AE093E062E771E00E94FD0A6401CC0CF1
:1002B000DD1C852D942D9C01790100E010E012C019
:1002C000F701619171917F018AE093E04AE050E08B
:1002D0000E94CF0A8AE093E06DE771E00E94FD0A78
:1002E0000F5F1F4FC016D10658F78AE093E00E94B7
:1002F000200A8AE093E00E94200AE2960FB6F89462
:10030000DEBF0FBECDBFCF91DF911F910F91FF9048
:10031000EF90DF90CF90BF90AF909F908F907F90A5
:100320006F905F904F9008956F927F928F929F92FF
:10033000AF92BF92CF92DF92EF92FF920F931F93F3
:1003400082E991E00E940602882321F182E991E08E
:100350000E941F025B016C0182E991E00E94280269
:100360003C0182E991E00E942D024C0182E991E07A
:100370000E9437028C0182E991E00E9432027C01E6
:10038000C601B501A30194010E94A00082E991E099
:100390000E9416021F910F91FF90EF90DF90CF9077
:1003A000BF90AF909F908F907F906F9008958AE05C
:1003B00093E040E855E260E070E00E94600882E966
:1003C00091E060E070E00E94AA060895FC012FEF22
:1003D0003FEF338322838AE090E09783868381E036
:1003E00080878EE591E095838483318320838CE33D
:1003F00090E09093800180937F011092DB01109236
:10040000DC011092DD011092DE01089520E0809160
:10041000DB019091DC01A091DD01B091DE0100973C
:10042000A105B10509F021E0822F08951092DB01AA
:100430001092DC011092DD011092DE0108956091AE
:10044000DB017091DC018091DD019091DE01089566
:100450008091DF019091E00108958091E1019091F8
:10046000E20108958091E3019091E401089585EE01
:1004700091E008952F923F924F925F926F927F92F8
:100480008F929F92AF92BF92CF92DF92EF92FF92A4
:100490000F931F93DF93CF93CDB7DEB762970FB65D
:1004A000F894DEBF0FBECDBF3C018091E501909175
:1004B000E6016FE170E00E943C0C4B017B0100E023
:1004C00010E020917F0130918001442737FD409555
:1004D000542FC801B7010E941D0C0E942C0B2AE06A
:1004E00037ED43E25CE30E94BA0B0E94000BA801C7
:1004F0009701220F331F441F551F2E0D3F1D401F14
:10050000511F59016A01A61AB70AC80AD90AAD8251
:10051000BE82CF82D8865B016C01A20EB31EC41EC0
:10052000D51EA982BA82CB82DC82AA24BB246501B3
:1005300021E030E03A87298717012801261A370A77
:10054000480A590AA8019701260F371F481F591F4B
:100550002F87388B498B5A8B7AC0E985FA85EE0F45
:10056000FF1FEB51FE4F808191819C0140E050E0E4
:10057000221633064406550658F58F859889A989B1
:10058000BA89281739074A075B0710F5E985FA8504
:10059000EE0FFF1FE951FE4F0190F081E02D7F012A
:1005A00000E010E0EB86FC860D871E878D819E8122
:1005B000AF81B8858E159F05A007B10748F48981E2
:1005C0009A81AB81BC81E816F9060A071B0778F10E
:1005D000ED80FE800F811885E216F30604071507EB
:1005E00058F589819A81AB81BC81281739074A0760
:1005F0005B0710F5E985FA85EE0FFF1FE951FE4F05
:1006000080819181A0E0B0E0281639064A065B0699
:1006100098F4EF84F88809891A898E159F05A00738
:10062000B10750F40894A11CB11CC11CD11CAA0C28
:10063000BB1CCC1CDD1C05C07A866986AA24BB24A1
:10064000650109851A850E5F1F4F1A87098729855D
:100650003A852615370508F480CFA60195015695F1
:1006600047953795279587E068167104C0F0209369
:10067000DB013093DC014093DD015093DE01769481
:1006800067947092E0016092DF019092E2018092A3
:10069000E10181E090E09093E4018093E30180E048
:1006A000211531054105510509F081E062960FB62B
:1006B000F894DEBF0FBECDBFCF91DF911F910F9198
:1006C000FF90EF90DF90CF90BF90AF909F908F9072
:1006D0007F906F905F904F903F902F9008952F9252
:1006E0003F924F925F926F927F928F929F92AF92C2
:1006F000BF92CF92DF92EF92FF920F931F93DF93FF
:10070000CF93CDB7DEB762970FB6F894DEBF0FBEBA
:10071000CDBF3C018091E5019091E6016AE070E077
:100720000E943C0C4B017B0100E010E020917F0116
:1007300030918001442737FD4095542FC801B701FF
:100740000E941D0C0E942C0B2AE037ED43E25CE373
:100750000E94BA0B0E94000BA8019701220F331FC1
:10076000441F551F59016A01A61AB70AC80AD90AB7
:10077000AD82BE82CF82D8865B016C01A20EB31E11
:10078000C41ED51EA982BA82CB82DC82AA24BB24D5
:10079000650121E030E03A87298717012801261AF0
:1007A000370A480A590AA8019701260F371F481F20
:1007B000591F2F87388B498B5A8B7AC0E985FA8568
:1007C000EE0FFF1FEB51FE4F808191819C0140E0B5
:1007D00050E0221633064406550658F58F85988951
:1007E000A989BA89281739074A075B0710F5E985EF
:1007F000FA85EE0FFF1FE951FE4F0190F081E02DC9
:100800007F0100E010E0EB86FC860D871E878D815E
:100810009E81AF81B8858E159F05A007B10748F46A
:1008200089819A81AB81BC81E816F9060A071B070A
:1008300078F1ED80FE800F811885E216F30604073B
:10084000150758F589819A81AB81BC812817390732
:100850004A075B0710F5E985FA85EE0FFF1FE9519E
:10086000FE4F80819181A0E0B0E0281639064A064B
:100870005B0698F4EF84F88809891A898E159F051C
:10088000A007B10750F40894A11CB11CC11CD11CD5
:10089000AA0CBB1CCC1CDD1C05C07A866986AA2468
:1008A000BB24650109851A850E5F1F4F1A870987CA
:1008B00029853A852615370508F480CFA6019501CC
:1008C000569547953795279587E068167104C0F0CF
:1008D0002093DB013093DC014093DD015093DE0176
:1008E000769467947092E0016092DF019092E20149
:1008F0008092E10182E090E09093E4018093E30133
:1009000080E0211531054105510509F081E062962D
:100910000FB6F894DEBF0FBECDBFCF91DF911F9110
:100920000F91FF90EF90DF90CF90BF90AF909F908E
:100930008F907F906F905F904F903F902F90089591
:100940002F923F924F925F926F927F928F929F92DF
:10095000AF92BF92CF92DF92EF92FF920F931F93CD
:10096000DF93CF93CDB7DEB76C970FB6F894DEBFA9
:100970000FBECDBF4C018091E5019091E60167E487
:1009800070E00E943C0C1B015B01CC24DD24209113
:100990007F0130918001442737FD4095542FC601D7
:1009A000B5010E941D0C0E942C0B2AE037ED43E29A
:1009B0005CE30E94BA0B0E94000B7B018C01D60104
:1009C000C50142E0880F991FAA1FBB1F4A95D1F7A6
:1009D0009C01AD012E193F09400B510B2D8B3E8B15
:1009E0004F8B588FA8019701280F391F4A1F5B1F93
:1009F000298B3A8B4B8B5C8BC601B5012BE030E029
:100A000040E050E00E941D0C9B01AC012E193F09F3
:100A1000400B510B2D873E874F87588BA8019701BC
:100A2000260F371F481F591F29873A874B875C8736
:100A3000D601C50133E0880F991FAA1FBB1F3A9545
:100A4000D1F78A0D9B1DAC1DBD1D9C01AD012E195A
:100A50003F09400B510B2D833E834F835887A801DC
:100A60009701280F391F4A1F5B1F29833A834B8345
:100A70005C83C601B50126E030E040E050E00E9412
:100A80001D0C2B013C014E185F08600A710A5701CA
:100A90006801A60EB71EC81ED91EA98EBA8ECB8EAF
:100AA000DC8EEE24FF24870161E070E070C0FB0162
:100AB000EE0FFF1FEB51FE4F808191819C0140E0C2
:100AC00050E08D899E89AF89B88D82179307A4075E
:100AD000B50720F5A988BA88CB88DC882A153B059C
:100AE0004C055D05D8F4FB01EE0FFF1FE951FE4FE9
:100AF00080819181A0E0B0E0AD84BE84CF84D888AD
:100B0000A816B906CA06DB0648F4A984BA84CB84C1
:100B1000DC848A159B05AC05BD0570F18D819E8135
:100B2000AF81B88582179307A407B50750F5A98050
:100B3000BA80CB80DC802A153B054C055D0508F5A5
:100B4000FB01EE0FFF1FE951FE4F80819181A0E074
:100B5000B0E0481659066A067B0698F4298D3A8D4E
:100B60004B8D5C8D82179307A407B50750F408944A
:100B7000E11CF11C011D111DEE0CFF1C001F111FBB
:100B800004C0B401EE24FF2487016E5F7F4F681517
:100B9000790508F48CCFA8019701569547953795AC
:100BA000279587E088169104C0F02093DB013093ED
:100BB000DC014093DD015093DE019694879490927E
:100BC000E0018092DF013092E2012092E10183E0B6
:100BD00090E09093E4018093E30180E021153105DA
:100BE0004105510509F081E06C960FB6F894DEBF1F
:100BF0000FBECDBFCF91DF911F910F91FF90EF906E
:100C0000DF90CF90BF90AF909F908F907F906F902C
:100C10005F904F903F902F900895CF92DF92EF9288
:100C2000FF920F931F93CF93DF930E9475076B0181
:100C30007C0180916D0290916E028601081B190B58
:100C4000109374020093730283E109381807C0F10E
:100C50002091E5013091E601C901885C9040801740
:100C6000910750F528533F4F0217130728F580913D
:100C70006B0290916C02019690936C0280936B02D0
:100C8000C0917102D09172022197D0937202C093E9
:100C90007102029789F4CE010E943A02882341F43E
:100CA000CE010E946F03882319F4CE010E94A00494
:100CB00010926C0210926B021092720210927102EA
:100CC00080917102909172028334910540F01092EC
:100CD00072021092710210926C0210926B0280915B
:100CE000710290917202FC01EE0FFF1FEB51FE4F5B
:100CF0001183008301969093720280937102C092D7
:100D00006D02D0926E02E0926F02F0927002DF915B
:100D1000CF911F910F91FF90EF90DF90CF900895AA
:100D2000FC01808191812FEF8F3F920791F010920B
:100D3000DB011092DC011092DD011092DE011092B5
:100D4000E0011092DF016DE076E041E050E00E94AA
:100D5000B0060895FC01718360830E949006089597
:100D6000823000F5E82FF0E0EE0FFF1FEB58FD4F4B
:100D700071836083882319F08130A1F408C08091C9
:100D800069008C7F842B80936900E89A0895809194
:100D90006900440F551F440F551F837F842B809398
:100DA0006900E99A08951F920F920FB60F921124CD
:100DB0002F933F934F935F936F937F938F939F9363
:100DC000AF93BF93EF93FF9380917502909176025A
:100DD000892B29F0E0917502F09176020995FF9137
:100DE000EF91BF91AF919F918F917F916F915F91A3
:100DF0004F913F912F910F900FBE0F901F9018951C
:100E00001F920F920FB60F9211242F933F934F937F
:100E10005F936F937F938F939F93AF93BF93EF9362
:100E2000FF938091770290917802892B29F0E091CD
:100E30007702F09178020995FF91EF91BF91AF9100
:100E40009F918F917F916F915F914F913F912F91E2
:100E50000F900FBE0F901F9018951F920F920FB614
:100E60000F9211242F933F938F939F93AF93BF9330
:100E700080917D0290917E02A0917F02B0918002CC
:100E8000309181020196A11DB11D232F2D5F2D37B9
:100E900020F02D570196A11DB11D20938102809352
:100EA0007D0290937E02A0937F02B0938002809196
:100EB000790290917A02A0917B02B0917C02019616
:100EC000A11DB11D8093790290937A02A0937B02B9
:100ED000B0937C02BF91AF919F918F913F912F91E1
:100EE0000F900FBE0F901F9018959FB7F894209108
:100EF000790230917A0240917B0250917C0286B552
:100F0000A89B06C08F3F21F02F5F3F4F4F4F5F4F91
:100F10009FBF542F432F322F2227280F311D411DF1
:100F2000511D82E0220F331F441F551F8A95D1F7B0
:100F3000B901CA010895789484B5826084BD84B5EE
:100F4000816084BD85B5826085BD85B5816085BDC4
:100F5000EEE6F0E0808181608083E1E8F0E01082DD
:100F6000808182608083808181608083E0E8F0E01E
:100F7000808181608083E1EBF0E080818460808308
:100F8000E0EBF0E0808181608083EAE7F0E080813F
:100F9000846080838081826080838081816080839F
:100FA0008081806880831092C100089508951F9207
:100FB0000F920FB60F9211242F933F934F938F935D
:100FC0009F93EF93FF938091C00082FD1DC04091DD
:100FD000C6002091C2023091C3022F5F3F4F2F7392
:100FE00030708091C4029091C5022817390771F0C2
:100FF000E091C202F091C302EE57FD4F408330935F
:10100000C3022093C20202C08091C600FF91EF91FB
:101010009F918F914F913F912F910F900FBE0F9005
:101020001F901895E0911603F0911703E05CFF4FB5
:101030008191919120813181821B930B8F739070EC
:10104000892B11F00E94D60708951F920F920FB6B8
:101050000F9211242F933F938F939F93EF93FF93BE
:1010600020910603309107038091080390910903B2
:101070002817390731F48091C1008F7D8093C1001A
:1010800014C0E0910803F0910903EA53FD4F208159
:10109000809108039091090301968F73907090934B
:1010A0000903809308032093C600FF91EF919F915D
:1010B0008F913F912F910F900FBE0F901F90189519
:1010C000AF92BF92DF92EF92FF920F931F93CF9355
:1010D000DF93EC017A018B01DD24403081EE58076B
:1010E00080E0680780E0780711F0DD24D39491E078
:1010F000A92EB12CEC89FD89DD2069F0C50108A07D
:1011000002C0880F991F0A94E2F7808360E079E0BB
:101110008DE390E005C0108260E874E88EE190E015
:10112000A80197010E94500C21503040404050408F
:10113000569547953795279580E12030380720F060
:10114000DD2011F0DD24D6CFE889F9893083EA89E2
:10115000FB89208319A2EE89FF89408121E030E0DC
:10116000C9010C8C02C0880F991F0A94E2F7482B22
:101170004083EE89FF894081C9010D8C02C0880F30
:10118000991F0A94E2F7482B4083EE89FF8940813A
:10119000C9010E8C02C0880F991F0A94E2F7482BF0
:1011A0004083EE89FF8980810F8C02C0220F331F9C
:1011B0000A94E2F7209528232083DF91CF911F9195
:1011C0000F91FF90EF90DF90BF90AF900895DC01FA
:1011D0001C96ED91FC911D97E05CFF4F21913191A0
:1011E00080819181281B390B2F733070C9010895BC
:1011F000DC011C96ED91FC911D97E05CFF4F208176
:101200003181E054F040DF01AE5BBF4F8D919C9186
:1012100011972817390719F42FEF3FEF07C08D9169
:101220009C91E80FF91F8081282F30E0C9010895B3
:10123000DC011C96ED91FC911D97E05CFF4F208135
:101240003181E054F040DF01AE5BBF4F8D919C9146
:1012500011972817390719F42FEF3FEF10C08D9120
:101260009C911197E80FF91F20818D919C91119706
:1012700001968F73907011969C938E9330E0C90104
:101280000895DC0191968C919197882339F05496BA
:10129000ED91FC915597808186FFF9CF91961C9234
:1012A0000895CF93DF93EC01EE85FF85E05CFF4F5F
:1012B00020813181E054F0402F5F3F4F2F73307019
:1012C000DF01AE5BBF4F8D919C91119728173907B5
:1012D000D1F3E05CFF4F80819181E054F040E80F52
:1012E000F91F6083EE85FF85E05CFF4F318320832B
:1012F000EE89FF89208181E090E00F8C02C0880F89
:10130000991F0A94E2F7282B208381E089A3EC89B6
:10131000FD8980818064808381E090E0DF91CF91BE
:10132000089510920D0310920C0388EE93E0A0E054
:10133000B0E080930E0390930F03A0931003B0933B
:10134000110385E891E090930B0380930A0382E8F0
:1013500092E0909317038093160386EC92E09093AB
:1013600019038093180385EC90E090931B038093FE
:101370001A0384EC90E090931D0380931C0380EC8F
:1013800090E090931F0380931E0381EC90E0909374
:1013900021038093200382EC90E0909323038093B9
:1013A000220386EC90E0909325038093240384E04D
:1013B0008093260383E08093270387E080932803AC
:1013C00085E08093290381E080932A030895CF93D9
:1013D000DF930E949B070E94D701C2E1D8E00E94E0
:1013E00094012097E1F30E941208F9CFCF92DF9287
:1013F000EF92FF920F931F93CF93DF937C016B01CA
:101400008A01C0E0D0E00FC0D6016D916D01D70117
:10141000ED91FC910190F081E02DC7010995C80F75
:10142000D91F015010400115110571F7CE01DF9150
:10143000CF911F910F91FF90EF90DF90CF90089583
:10144000EF92FF920F931F938C01DC01ED91FC91C1
:101450000190F081E02D6DE009957C01D801ED91BE
:10146000FC910190F081E02DC8016AE009959C0192
:101470002E0D3F1DC9011F910F91FF90EF90089510
:10148000CF93DF93EC016115710519F420E030E092
:101490000FC0DB010D900020E9F71197A61BB70BD9
:1014A000E881F9810280F381E02DAD0109959C016D
:1014B000C901DF91CF9108954F925F927F928F92F1
:1014C0009F92AF92BF92CF92DF92EF92FF920F93D3
:1014D0001F93DF93CF93CDB7DEB7A1970FB6F894E4
:1014E000DEBF0FBECDBF2C01742ECB01223008F41D
:1014F0002AE019A231E2C32ED12CCC0EDD1E822EA1
:101500009924AA24BB24672D752FA50194010E945C
:10151000500C79018A01C801B701A50194010E940C
:101520001D0C472D461B0894C108D1084A3014F4FD
:10153000405D01C0495CF6014083E114F1040105FE
:10154000110521F07E2C5F2DC801DDCFC201B6014F
:101550000E94400AA1960FB6F894DEBF0FBECDBF21
:10156000CF91DF911F910F91FF90EF90DF90CF907F
:10157000BF90AF909F908F907F905F904F90089515
:10158000DC012115310541F4ED91FC910190F081D0
:10159000E02D642F099508950E945C0A0895EF924A
:1015A000FF920F931F939A017B0100E010E0B801B6
:1015B000A7010E94C00A1F910F91FF90EF9008951C
:1015C000CF92DF92EF92FF920F931F936C017B01FA
:1015D0009A0100E010E0B801A7010E94C00A8C0146
:1015E000C6010E94200A080F191FC8011F910F9100
:1015F000FF90EF90DF90CF9008950E94400A0895E9
:1016000098D088F09F5790F0B92F9927B751A0F044
:10161000D1F0660F771F881F991F1AF0BA95C9F786
:1016200012C0B13081F09FD0B1E008959CC0672F07
:10163000782F8827B85F39F0B93FCCF38695779536
:101640006795B395D9F73EF490958095709561951F
:101650007F4F8F4F9F4F0895E89409C097FB3EF44A
:1016600090958095709561957F4F8F4F9F4F9923EF
:10167000A9F0F92F96E9BB279395F695879577956D
:101680006795B795F111F8CFFAF4BB0F11F460FF2D
:101690001BC06F5F7F4F8F4F9F4F16C0882311F085
:1016A00096E911C0772321F09EE8872F762F05C099
:1016B000662371F096E8862F70E060E02AF09A9534
:1016C000660F771F881FDAF7880F9695879597F929
:1016D000089597F99F6780E870E060E008959FEFB4
:1016E00080EC089500240A941616170618060906B9
:1016F000089500240A941216130614060506089588
:10170000092E0394000C11F4882352F0BB0F40F40F
:10171000BF2B11F460FF04C06F5F7F4F8F4F9F4F4F
:10172000089557FD9058440F551F59F05F3F71F0D1
:101730004795880F97FB991F61F09F3F79F0879538
:101740000895121613061406551FF2CF4695F1DFC1
:1017500008C0161617061806991FF1CF8695710551
:10176000610508940895E894BB2766277727CB0185
:1017700097F908950BD0C4CFB5DF28F0BADF18F081
:10178000952309F0A6CFABCF1124EECFCADFA0F38B
:10179000959FD1F3950F50E0551F629FF001729F06
:1017A000BB27F00DB11D639FAA27F00DB11DAA1F25
:1017B000649F6627B00DA11D661F829F2227B00D72
:1017C000A11D621F739FB00DA11D621F839FA00DFD
:1017D000611D221F749F3327A00D611D231F849F4D
:1017E000600D211D822F762F6A2F11249F575040A4
:1017F0008AF0E1F088234AF0EE0FFF1FBB1F661F3F
:10180000771F881F91505040A9F79E3F510570F0F7
:1018100060CFAACF5F3FECF3983EDCF386957795D7
:101820006795B795F795E7959F5FC1F7FE2B880FF2
:10183000911D9695879597F90895629FD001739FA2
:10184000F001829FE00DF11D649FE00DF11D929F5C
:10185000F00D839FF00D749FF00D659FF00D99279B
:10186000729FB00DE11DF91F639FB00DE11DF91FBF
:10187000BD01CF0111240895AA1BBB1B51E107C074
:10188000AA1FBB1FA617B70710F0A61BB70B881F10
:10189000991F5A95A9F780959095BC01CD0108959F
:1018A000A1E21A2EAA1BBB1BFD010DC0AA1FBB1F64
:1018B000EE1FFF1FA217B307E407F50720F0A21BD6
:1018C000B30BE40BF50B661F771F881F991F1A9443
:1018D00069F760957095809590959B01AC01BD016D
:1018E000CF010895EE0FFF1F0590F491E02D0994AC
:1018F000F894FFCF556E6B6E6F776E20656E636FD9
:1019000064696E672E00446563696D616C3A2000FE
:10191000202800426974292042696E6172793A2058
:1019200000205472692D53746174653A20006E6F03
:1019300074206170706C696361626C650020507521
:101940006C73654C656E6774683A2000206D69633E
:10195000726F7365636F6E6473002050726F746F83
:10196000636F6C3A200052617720646174613A20A1
:10197000002C003C00000000005109F609E708189F
:1019800009F808410900446563696D616C3A2000FB
:10199000202800426974292042696E6172793A20D8
:1019A00000205472692D53746174653A20006E6F83
:1019B00074206170706C696361626C6500205075A1
:1019C0006C73654C656E6774683A2000206D6963BE
:1019D000726F7365636F6E6473002050726F746F03
:1019E000636F6C3A200052617720646174613A2021
:1019F000002C003C00000000005109F609E708181F
:101A0000D801DA962D913D914D915C91DD97261785
:101A100037074807590728F0F6018081833009F01D
:101A200000CFC2010E949F1AF80184819581A6818E
:101A3000B7810196A11DB11D84839583A683B783C9
:101A4000C3010F900F900F900F90CF91DF911F91D6
:101A50000F91FF90EF90DF90CF90BF90AF909F904D
:101A60008F907F906F905F904F903F902F90089550
:101A7000CF92DF92EF92FF920F931F93CF93DF935A
:101A8000EC01D62EC72E1AA21BA21CA21DA21EA2BA
:101A90001FA218A619A61AA61BA61CA61DA61EAA3A
:101AA0001FAA18AE19AE2AAF3BAF4CAF5DAFEE9692
:101AB000E882F9820A831B83EE978E01085F1F4F2D
:101AC00086E0F80111928A95E9F7CE010E94570A43
:101AD000D8012D2D3C2DC901FC0186E001900D920D
:101AE0008150E1F7CA5BDF4F1882C654D040CE0167
:101AF0000E94B50BDF91CF911F910F91FF90EF9056
:101B0000DF90CF9008959C01FB0182819381A48195
:101B1000B581F90182839383A483B58317821682EA
:101B20000895CF93DF93FB0101C031968081882314
:101B3000E1F7EB01A0E0B0E020E030E021C06E3240
:101B400061F42F3F310509F07CF5FA01EA0FFB1F24
:101B50002283119620E030E012C0C901E3E0880F33
:101B6000991FEA95E1F7220F331F820F931F262F4B
:101B7000332727FD309520533040280F391F2196F9
:101B80006881662319F0A430B105CCF22F3F3105EE
:101B900009F054F4A430B1053CF4A40FB51F12961B
:101BA0002C9321E030E002C020E030E0C901DF9159
:101BB000CF9108950F938FEA92E060E040E020E03B
:101BC00000E00E9427360F9108952F923F924F9286
:101BD0005F926F927F928F929F92AF92BF92CF92BD
:101BE000DF92EF92FF920F931F93DF93CF93CDB7C6
:101BF000DEB769970FB6F894DEBF0FBECDBF2C01DC
:101C00008B011A010E94E5323B014C01F8E0AF2E36
:101C1000B12CA40CB51C780100E010E014C00E94A7
:101C2000E5326619770988099909E616F706080763
:101C3000190718F42FEF3FEF10C162E370E080E066
:101C400090E00E941933C5010E9420191816190648
:101C500034F7F201C280D380E480F5808E01085F02
:101C60001F4FC801B5010E94EC18F80182819381D1
:101C7000A481B581C816D906EA06FB0609F0EBC0B7
:101C8000C5010E947B18C59709F0E5C000C18E010F
:101C9000025F1F4FC501B8014CE050E00E94581987
:101CA000F801528143815B834A83F20126813781A7
:101CB0008E859F852817390711F457FD06C0C50189
:101CC0000E9412192CEF3FEFC8C04F705270452B85
:101CD00031F0C5010E9412192BEF3FEFBEC0F80191
:101CE000568047804114510441F0882499246801AA
:101CF0003E010894611C711C28C0C5010E94121984
:101D00002AEF3FEFAAC0C501B30141E050E00E94B5
:101D100058198981882321F408C0C5010E9432180E
:101D20008981815089838F5FC1F78981882359F721
:101D300000E010E0C5010E9432180F5F1F4F043011
:101D40001105C1F70894811C911CF601F480E5800F
:101D50008E149F04C0F2CC24DD24C501BE016F5F48
:101D60007F4F41E050E00E9458199981892F807C73
:101D700061F4992321F40DC0C5010E9432188981B4
:101D8000815089838F5FC1F704C0C5010E9432185A
:101D900019828981882309F7C501BE016C5F7F4FD5
:101DA00042E050E00E945819C501BE016A5F7F4FB2
:101DB00042E050E00E94581900E010E0C5010E9486
:101DC00032180F5F1F4F04301105C1F7C501BE0166
:101DD0006E5F7F4F42E050E00E945819FC80ED801A
:101DE000F1E0EF16F10419F59E808F8081E08816EE
:101DF0009104E9F49A818B81049731F0C5010E9426
:101E0000121927EF3FEF29C0E2E0F0E02E0E3F1E4F
:101E1000C501B10144E050E00E94581921E030E0D2
:101E20001CC0C5010E9432180F5F1F4F02C000E0A6
:101E300010E07A806B800615170598F30894C11C92
:101E4000D11CC414D50408F488CFC5010E9412190E
:101E500026EF3FEF02C02EEF3FEFC90169960FB6A4
:101E6000F894DEBF0FBECDBFCF91DF911F910F91D0
:101E7000FF90EF90DF90CF90BF90AF909F908F90AA
:101E80007F906F905F904F903F902F900895C50185
:101E90000E9406190C970CF0FACE2DEF3FEFDDCF24
:101EA0006F927F928F929F92AF92BF92CF92DF926A
:101EB000EF92FF920F931F93DF93CF9300D00F9277
:101EC000CDB7DEB78C01F62EE72E0E94E532F80181
:101ED00077836683B8E0CB2ED12CC00ED11E0A5F6B
:101EE0001F4FC601B80142E050E00E948D1981E009
:101EF00090E09B838A83A2E08A2E912C8C0E9D1EFB
:101F0000C601B40142E050E00E948D1980E091E0EA
:101F10009B838A83C601B40142E050E00E948D1980
:101F20001B821A82C601B40142E050E00E948D1962
:101F3000C601B40142E050E00E948D19C601B4010F
:101F400042E050E00E948D192F2D3E2DC9018C01D9
:101F50007C013E010894611C711C20C00894E11CA6
:101F6000F11CF7018081882311F08E32B9F75701F7
:101F7000A01AB10A1A141B0474F48E2D801B8983D5
:101F8000C601B30141E050E00E948D19C601B801BD
:101F9000A5010E948D1987010F5F1F4FF7018081F6
:101FA000882311F07801DDCF1982C601BE016F5F71
:101FB0007F4F41E050E00E948D1900E011E01B834B
:101FC0000A83C601B40142E050E00E948D191B83D0
:101FD0000A83C601B40142E050E00E948D1981E0FD
:101FE00090E00F900F900F90CF91DF911F910F9184
:101FF000FF90EF90DF90CF90BF90AF909F908F9029
:102000007F906F9008958F929F92AF92BF92CF92E0
:10201000DF92EF92FF920F931F93DF93CF9300D045
:1020200000D000D0CDB7DEB76C017B014A010E9421
:10203000910D892B19F001E010E067C0F6012281B3
:102040003381448155818091B1029091B202A09177
:10205000B302B091B402281739074A075B0719F495
:102060000EEF1FEF52C018E0A12EB12CAC0CBD1C1E
:102070000E94E5329B01AC012F70307020503C4F24
:10208000C501B9010E94711A813019F000E010E019
:102090003CC085E092E09A838983F6018281938136
:1020A000A481B5818B839C83AD83BE83C501BE01B2
:1020B0006F5F7F4F45E350E00E94D7198C01009776
:1020C00009F1C601B7010E94500F8C010097D1F0B1
:1020D000C5010E94A8198C010097A1F0EE24FF24ED
:1020E000C60168E873E1A4010E94E50D8C01089423
:1020F000E11CF11CF3E0EF16F10421F08FEF0F3F2C
:10210000180771F3C5010E949F1AC80126960FB6E1
:10211000F894DEBF0FBECDBFCF91DF911F910F911D
:10212000FF90EF90DF90CF90BF90AF909F908F90F7
:102130000895DC01ED91FC91008CF18DE02D099565
:1021400091E089270895FC011382128288EE93E0C2
:10215000A0E0B0E084839583A683B7838FE991E004
:1021600091838083158614860895DC011C96ED9179
:10217000FC911D97309711F480E0089581818823A8
:1021800011F081E00895808190E024E09695879594
:102190002A95E1F781700895FB01DC011C962D91D1
:1021A0003C911D972115310559F0648575856115A0
:1021B000710531F080E02617370719F481E00895A2
:1021C00080E00895DF93CF930F92CDB7DEB7FC0187
:1021D000A081B18150962D913C915197BE016F5FC6
:1021E0007F4F41E050E0F901099597FF03C02FEFC1
:1021F0003FEF03C08981282F30E0C9010F90CF91B4
:10220000DF9108950F9389EF92E060E040E020E0D5
:1022100000E00E9427360F9108951F93CF93DF931C
:10222000EC0110E088810E94F82A19921F5F153096
:10223000C9F7DF91CF911F910895CF93DF93EC0100
:10224000E881F9810688F789E02D0995882329F02E
:102250008C859D8501960E940D11DF91CF91089587
:10226000CF93DF93EC0188810E94F82AFE0190E071
:10227000818181939F5F9430D9F71C82DF91CF9148
:102280000895CF93DF93E5EBF2E020E030E0922F6A
:10229000A90164E0440F551F6A95E1F7420F531FEF
:1022A000DA01AB54BD4F8081882361F490619C9327
:1022B000CA018A549D4FFC0180E1EF0119928A9571
:1022C000E9F708C02F5F3F4F719624303105F9F6CA
:1022D000A0E0B0E0CD01DF91CF910895FF920F9380
:1022E0001F93CF93DF938C01C0E0D0E0FF24F8016F
:1022F00081810E940A27C80FD91FF3940F5F1F4FD7
:10230000F5E0FF16A1F7CE01DF91CF911F910F915C
:10231000FF900895CF93DF93EC01E881F98106885F
:10232000F789E02D0995882319F420E030E005C0F5
:102330008C859D850E946E119C01C901DF91CF9112
:102340000895DF92EF92FF920F931F93CF93DF9345
:10235000E091AB06F091AC06E48CF58CE114F1044D
:1023600081F48091A60686FFDFC00E9441117C01A6
:10237000009709F4D9C0E091AB06F091AC06958FB7
:10238000848F8091A60681FF3DC080919E0690912A
:102390009F06892BB9F1F7018081807699F5E701D5
:1023A000DD2489818823E9F480919E0690919F061F
:1023B0000E94462B89838823A1F02091A9063091A1
:1023C000AA062953374000919E0610919F0660E0AF
:1023D00070E04091FF020E94BE29F4E0DF1691F404
:1023E0000AC0D394219685E0D816D9F680910203CD
:1023F0008E7F80930203E091AB06F091AC06818D55
:102400008061818FF701808187FF0EC08F77808385
:102410008091A60682608093A606E091AB06F091BB
:10242000AC06818D8F7E818F8091A60684FD02C0CF
:1024300087FF1EC0C70106960E940D11F70181811A
:10244000882369F0E091AB06F091AC068481958118
:10245000F7019783868380818064808302C0F701BF
:102460001082E091AB06F091AC06158E148E5CC024
:1024700080FF04C0C70106960E9430118091A60615
:102480008C70C9F1F70196819923A9F1878188237E
:1024900061F4C385D485209709F448C0892F60E092
:1024A00070E0AE010E94332B06C0892F0E940A27DC
:1024B000EC010097D9F12091A90689E397E0281B48
:1024C00020930103CE01820F911D0E94462B809321
:1024D0000003882359F16091010370E0F701468100
:1024E00020E030E08E010E94BE29809102038260CC
:1024F000809302031BC0F701808185FF15C0868190
:10250000882359F41082E091AB06F091AC06158E49
:10251000148E80E18093A60607C0E091AB06F0918F
:10252000AC06818D8061818FC0E0D0E08091A906EA
:102530009091AA06BE010E94591CD0939F06C09399
:102540009E06DF91CF911F910F91FF90EF90DF904A
:1025500008950F931F93DF93CF930F92CDB7DEB7FC
:102560008C01DC01ED91FC910688F789E02D09953D
:102570008823A9F0D8011C96ED91FC911D978181CB
:10258000882369F060E070E0AE014F5F5F4F21E0AB
:1025900030E00E943B288981282F30E002C02FEFD5
:1025A0003FEFC9010F90CF91DF911F910F910895D7
:1025B000AF92BF92CF92DF92EF92FF920F931F9351
:1025C000CF93DF938C015B016A01DC01ED91FC91FB
:1025D0000688F789E02D0995882319F44FEF5FEFFE
:1025E0006EC0D8011C96ED91FC911D9781818823C6
:1025F00019F440E050E063C07601D8011C96ED91DB
:10260000FC911D97A6014E195F094A0D5B1D818142
:1026100060E070E097010E943B28EC01D8011C9615
:10262000ED91FC911D9781810E940A27D8011C968B
:10263000ED91FC911D97C817D907B9F5EC1AFD0A61
:10264000CF0101960E943011F801A485B5854C9107
:10265000242F30E0C9018F70FC0155E0EE0FFF1F01
:102660005A95E1F7880F991FE81BF90BE355F94FCD
:10267000818D84FF06C020763070232B11F44068D2
:102680004C93D8011C96ED91FC911D978181882374
:1026900089F4808186FF05C010821D961C921E92CF
:1026A0001C97A6014E195F090AC08181BE010E94D4
:1026B0001C2B04C0E114F10409F09FCFA601CA014C
:1026C000DF91CF911F910F91FF90EF90DF90CF900E
:1026D000BF90AF9008950F931F938C010E948316B3
:1026E000D8011C96ED91FC911D97309711F480E074
:1026F00006C0808186FF02C08181811181E01F9127
:102700000F910895CF93DF93EC01EC85FD85309711
:1027100081F08081882369F0CF0101960E940D111C
:10272000EC85FD85808186FF02C0108202C0806238
:1027300080831D861C860E948316DF91CF910895A9
:10274000AF92BF92CF92DF92EF92FF921F93CF93FF
:10275000DF93EC015B016A017A010E9483162097E6
:1027600009F44FC08881807609F04BC0FE0191E0EA
:102770008781882319F4192F115005C09F5F319666
:102780009530B1F714E0FE01E10FF11D8681882339
:1027900061F480E092E00E94462BFE01E10FF11D02
:1027A00086838823D1F21C861B86FE01E10FF11D72
:1027B0006B857C85A6014E195F094A0D5B1D8681DC
:1027C00097010E94C327E81AF90A2B853C85280F38
:1027D000391F3C872B871E141F042CF4143009F476
:1027E000BCCF1F5FD6CF0E94E532665F7F4F8F4F11
:1027F0009F4F6D877E878F87988B96012E193F0993
:1028000002C02FEF3FEFC901DF91CF911F91FF90E1
:10281000EF90DF90CF90BF90AF900895FC0184853A
:1028200095850E94A0130895DF93CF930F92CDB7A3
:10283000DEB76983FC0184859585BE016F5F7F4F9C
:1028400041E050E00E94A0130F90CF91DF910895D6
:102850008F929F92AF92BF92CF92DF92EF92FF92B0
:102860000F931F93DF93CF93CDB7DEB7A8970FB623
:10287000F894DEBF0FBECDBF5C018B014A016DE055
:10288000E62EF12CEC0EFD1EC7010E949536CE01FE
:1028900045960E94C01A6E010894C11CD11CC60145
:1028A0000E949536C70163E073E00E94830DC70163
:1028B000B801A6010E9403109C0181309105C9F462
:1028C000D501ED91FC910484F585E02D85E092E041
:1028D00098878F838B819C81AD81BE8189879A8700
:1028E000AB87BC87C501BE01695F7F4FA401099515
:1028F0009C01C901A8960FB6F894DEBF0FBECDBFEC
:10290000CF91DF911F910F91FF90EF90DF90CF90CB
:10291000BF90AF909F908F900895CF92DF92EF92EB
:10292000FF920F931F93DF93CF9300D000D0CDB7CA
:10293000DEB76C018B017A01DC01ED91FC9102881C
:10294000F389E02D0995F801328120E0838190E040
:10295000822B932B292F3327982F8827282B392B2D
:102960003A832983348120E0858190E0822B932B68
:10297000292F3327982F8827282B392B3C832B830B
:10298000C7010E94551CBC01CE0101960E94BD1BCF
:102990008C010097A1F41BC00E948316D8015996A0
:1029A0008C9159978F70833051F45C968D919C91E6
:1029B0005D97F6019587848721E030E00AC0D80151
:1029C00059968C9190E08F709070892B29F720E0B8
:1029D00030E0C9010F900F900F900F90CF91DF91D1
:1029E0001F910F91FF90EF90DF90CF900895FC0121
:1029F00025E032E0318320832091050330910603E6
:102A00004091070350910803228333834483558305
:102A100008950F931F93FC018B01DA01B901928194
:102A200080E0438150E0482B592B348120E08581A0
:102A300090E0822B932B252F3327542F4427242BD0
:102A4000352B3093360720933507292F3327982FBE
:102A50008827282B392B3093380720933707129675
:102A60009C91129780E013964C91139750E0482B5D
:102A7000592B14963C91149720E015968C9190E078
:102A8000822B932B252F3327542F4427242B352B90
:102A900030932E0720932D07292F3327982F88272F
:102AA000282B392B3093300720932F07FB0192817D
:102AB00080E0438150E0482B592B348120E0858110
:102AC00090E0822B932B252F3327542F4427242B40
:102AD000352B3093320720933107292F3327982F36
:102AE0008827282B392B3093340720933307F8019C
:102AF00082819381A481B58180930503909306031D
:102B0000A0930703B09308031F910F9108959C01B0
:102B100041505040460F571FFB010EC0708160E0CE
:102B20008181DB01A80FB11D2A0F3B1F2A173B072C
:102B300010F42F5F3F4F3296E417F50778F3E41750
:102B4000F50749F4908180E0280F391F28173907CD
:102B500010F42F5F3F4FC90108950F9380E193E078
:102B600060E040E020E000E00E94273683E093E050
:102B70000E9495360F910895EF92FF921F93CF9385
:102B8000DF93182F80914A07E82EFF248CEE9FEFE9
:102B9000E80EF91E9091490780E0E80EF91EC70182
:102BA000810F911D63E577E048E050E00E948715B2
:102BB000113111F448E005C04091670746954695EC
:102BC0004C73C42FD0E06BE577E0AE010E9487150F
:102BD000CE15DF0548F4EC1AFD0A60910003A296B9
:102BE000AE0197010E947028009719F42FEF3FEF74
:102BF00003C00E94551C9C01C901DF91CF911F9118
:102C0000FF90EF90089581E10E94BC15089586E041
:102C10000E94BC15089580E090E067E477E044E10D
:102C200050E00E948715009719F42FEF3FEF03C083
:102C30000E94551C9C01C90108950E940B1608951D
:102C40000F931F938C010E94E53266507F4F8F4F88
:102C50009F4F60930B0370930C0380930D0390932D
:102C60000E03C8010E94522AF801808180938503D7
:102C700081818093860382818093870383818093FF
:102C80008803848180938903858180938A030E94CD
:102C90007F1B0E94F5261F910F91089580910203DA
:102CA00081FF11C0209101038091000360E070E07A
:102CB00049E357E030E00E94C327809102038D7FF3
:102CC0008093020314C080919E0690919F060E94FB
:102CD000462B809300038823A9F020919E06309113
:102CE0009F0660E070E049E357E00E94C3278091AF
:102CF00000030E94F629809100030E94F82A109296
:102D0000000381E00895BF92CF92DF92EF92FF928D
:102D10000F931F93CF93DF938091FF02882321F4B9
:102D20000E94E8288093FF029091FF02992309F402
:102D300048C081E080930203892F0E940A27909364
:102D40009F0680939E06892B81F18091FF0260E0AF
:102D500070E049E357E022E630E00E943B28809192
:102D60004507909146078830910591F48091FF02C4
:102D7000809300030E94092581E00E946F1C8091CE
:102D80009E0690919F06892B81F00E94F3250BC02F
:102D90008850964051F40E943D2580919E06909166
:102DA0009F06892B11F00E944E168091FF02882306
:102DB00041F08091020380FF04C00E945F281092BE
:102DC000FF020E94E5327B018C01BB2480910B0342
:102DD00090910C03A0910D03B0910E03A8019701EF
:102DE000281B390B4A0B5B0B57FD02C0BB24B39465
:102DF00069ECC62E66E0D62EC0E0D0E09E01220F20
:102E0000331FCE0145E0880F991F4A95E1F7821BD9
:102E1000930B8355994F9093AC068093AB06BB20E0
:102E200011F082E010C0D601ED91FC918585968568
:102E3000A785B089A8019701281B390B4A0B5B0BAA
:102E400057FD0DC083E00E946F1C80919E069091FB
:102E50009F06892B21F00E94F3250E944E16219691
:102E60004EE150E0C40ED51EC430D10539F6BB206A
:102E7000B9F18AEF90E0A0E0B0E0E80EF91E0A1F79
:102E80001B1FE0920B03F0920C0300930D031093B1
:102E90000E03C8EAD7E000E010E0BBE0EB2EF12C17
:102EA0000E9DC0010F9D900D1E9D900D1124815609
:102EB000984F9093A8068093A70685E00E946F1C08
:102EC00080919E0690919F06892B21F0888199819F
:102ED0000E945E180F5F1F4F2B960430110501F7FB
:102EE000DF91CF911F910F91FF90EF90DF90CF90E6
:102EF000BF9008958F929F92AF92BF92CF92DF9230
:102F0000EF92FF920F931F93DF93CF93CDB7DEB76E
:102F100068970FB6F894DEBF0FBECDBF8B018091CE
:102F20001603882371F486E193E00E94AE36892B64
:102F300041F085E693E00E94C01A86E193E00E948A
:102F4000B8368EE193E090930A0380930903C80199
:102F50000E9420168091090390910A03B80120E68F
:102F60003AEE40E050E0B0EAEB2EBFE0FB2E012D40
:102F7000112D0E94380D4C0181E08816910499F5BD
:102F80006091090370910A035E010894A11CB11CB1
:102F9000C5010E94F507A7E0CA2ED12CCC0EDD1E7C
:102FA0006091090370910A03C6010E94D407FDE0F5
:102FB000EF2EF12CEC0EFD1E6091090370910A03B7
:102FC000C7010E94DF078E010D5E1F4F609109034C
:102FD00070910A03C8010E94EA07C501B601A70162
:102FE00098010E940915C40168960FB6F894DEBFD7
:102FF0000FBECDBFCF91DF911F910F91FF90EF904A
:10300000DF90CF90BF90AF909F908F9008950F93D7
:1030100089E793E060E040E020E000E00E9427368E
:103020000F910895DC01ED91FC91008CF18DE02D64
:1030300009950895DF93CF930F92CDB7DEB7FC01CA
:103040006983A081B18112962D913C911397BE01A5
:103050006F5F7F4F41E050E0F90109950F90CF91EC
:10306000DF910895DF93CF930F92CDB7DEB7FC01C8
:10307000A081B18158962D913C915997BE016F5F07
:103080007F4F41E050E0F9010995181619061CF030
:103090002FEF3FEF03C08981282F30E0C9010F9047
:1030A000CF91DF9108950F938FE793E060E040E0C8
:1030B00020E000E00E9427360F910895CF93DF9320
:1030C000EC010E94F32580919E0690919F068A97BD
:1030D00031F410920003809102038D7F05C01D82A0
:1030E0001C82809102038260809302030E944E162C
:1030F000DF91CF910895DC011C96ED91FC911D9715
:10310000309719F420E030E005C0868197810E9455
:10311000551C9C01C9010895EF92FF920F931F93D4
:10312000CF93DF93E091A706F091A806C185D285E1
:10313000209709F44AC08091A60681FF2FC08A819A
:10314000882361F580915B0790915C079783868364
:103150008091530790915407918380838091550704
:10316000909156079383828380915F0790916007C7
:103170000E94551C08970E94462BE82E8A838823BC
:1031800069F0F090FF020E940A278C018E2D60E00A
:1031900070E04F2D2AE230E00E94BE298091A60601
:1031A00083FF13C08D81882381F08C81809300037D
:1031B0008AE280930103688179816A52704080912C
:1031C000A9069091AA060E94591CDF91CF911F91E8
:1031D0000F91FF90EF900895FF920F931F93182F78
:1031E000F92EFB010484F585E02D309739F06081DC
:1031F0004181228103810E94273602C00E949536B8
:10320000812F9F2D1F910F91FF9008950F931F9372
:103210008C010E948316F80181890E940A271F9160
:103220000F9108950F931F938C010E948316F8014C
:1032300081890E94F82AF801118A1F910F9108953F
:103240000F931F938C010E948316F80181890E94BD
:10325000F82AF8018089818B108A0E940A271F9121
:103260000F9108950F931F93DF93CF930F92CDB7D4
:10327000DEB78C010E948316F8018189882379F0DA
:1032800060E070E0AE014F5F5F4F21E030E00E94F0
:103290003B28019721F48981282F30E002C02FEFCD
:1032A0003FEFC9010F90CF91DF911F910F910895CA
:1032B000EF92FF920F931F93CF93DF938C01EB015B
:1032C0007A010E948316F8018189882319F460E04D
:1032D00070E01BC060E070E0AE0197010E943B28E7
:1032E000EC01F80181890E940A27C817D90739F42F
:1032F000F80181890E94F82AF801118A05C0F801B5
:103300008189BE010E941C2BBE01CB01DF91CF91B0
:103310001F910F91FF90EF900895CF93DF93EC01F1
:10332000FB019A018A89882319F420E030E00CC05F
:103330006E857F85AF010E94C3279C018E859F8586
:10334000820F931F9F878E87C901DF91CF910895C8
:10335000CF93DF93EC018C859D85892B11F19A89A0
:103360009923F9F081E08B8B4E855F85892F60E092
:1033700070E00E94332B8C859D859093A8068093E6
:10338000A70685E00E946F1C80919E0690919F0683
:10339000892B39F0CE010E960E945E1821E030E0B4
:1033A00002C020E030E0C901DF91CF910895CF92B3
:1033B000DF92EF92FF920F931F93DF93CF9300D092
:1033C00000D0CDB7DEB78C017B016A010E94831665
:1033D000F70182819381A481B5810097A105B10590
:1033E00009F452C0C114D10409F44EC0328120E066
:1033F000838190E0822B932B292F3327982F8827C6
:10340000282B392B3A832983348120E0858190E071
:10341000822B932B292F3327982F8827282B392B62
:103420003C832B83D8011C96ED90FC901D97E114F2
:10343000F104A1F0C6010E94551CF7019783868311
:10344000D8011C96ED91FC911D9789819A819183F9
:1034500080838B819C819383828316C0C6010E94E6
:10346000551CBC01CE0101960E94EB23FC01D80142
:103470001D969C938E931C97009719F1025F1F4F26
:10348000128701870E501040F80184859585892B9D
:10349000C1F082898823A9F486E096E00E94462B39
:1034A000D80152968C9352972AE230E01F963C93B3
:1034B0002E931E9720E030E0882329F021E030E0B1
:1034C00002C020E030E0C9010F900F900F900F90E4
:1034D000CF91DF911F910F91FF90EF90DF90CF90F0
:1034E0000895EF92FF920F931F93CF93DF93EC0118
:1034F0007B018C859D85892B41F480E090E060E024
:1035000070E00E94EB239D878C870C851D8501153B
:10351000110511F480E00CC0C7010E94551CF80190
:1035200095838483EC85FD852E96D287C18781E0C3
:10353000DF91CF911F910F91FF90EF900895CF935E
:10354000DF93EC01EC85FD853097B9F0158214828C
:10355000128611861D861C8689890E94F82A888910
:103560000E94F82A8A890E94F82ACE010E96FC0150
:1035700086E0DF011D928A95E9F7DF91CF910895EA
:10358000FC011382128288EE93E0A0E0B0E0848315
:103590009583A683B7838FEB91E091838083158613
:1035A00014863E9686E011928A95E9F708956F9207
:1035B0007F928F929F92AF92BF92CF92DF92EF92C3
:1035C000FF920F931F93DF93CF93CDB7DEB7AE97E4
:1035D0000FB6F894DEBF0FBECDBF4C015B013A01C0
:1035E000E3E1EE2EF12CEC0EFD1EC7010E94953694
:1035F000CE014B960E94C01A6E010894C11CD11CCA
:10360000C6010E9495368E01095F1F4FC8016FE009
:1036100073E00E94F714C701B8010E94830DC7012F
:10362000B501A6010E9403109C0181309105C9F4E7
:10363000D401ED91FC910088F189E02D85E092E0C4
:103640009E878D878B819C81AD81BE818F87988B72
:10365000A98BBA8BC401BE01635F7F4FA30109959B
:103660009C01C901AE960FB6F894DEBF0FBECDBF68
:10367000CF91DF911F910F91FF90EF90DF90CF904E
:10368000BF90AF909F908F907F906F900895FC01B6
:103690005381560F5093A506272F33274281420F9F
:1036A0004093A406A181A093A306E081E093A20623
:1036B000842F90E08217930748F48A2F8F5F8093BE
:1036C000A306882319F4EF5FE093A206852F90E00C
:1036D00070708617970790F4842F8F5F8093A406ED
:1036E000882361F48091A3068F5F8093A3068823CB
:1036F00029F48091A2068F5F8093A206089580E04E
:1037000009C0E82FF0E0EE0FFF1FEB5DF84F1182CC
:1037100010828F5F8430A8F320E010C0822F90E0E9
:10372000FC0145E0EE0FFF1F4A95E1F7880F991F56
:10373000E81BF90BE355F94F118E2F5F243070F31E
:1037400080E094E0909392038093910320E04BE01B
:1037500050E00EC0822F90E0849FF001859FF00D15
:10376000949FF00D1124E156F84F158214822F5FBB
:10377000243080F3209393030895CF93DF93EC01DB
:103780004091910350919203BEE14F5F5F4F8DE7EF
:103790004030580710F040E050E1342F252FA0E0D2
:1037A0000EC0AB9FF0011124E355F94F818D8823A2
:1037B00029F0848195818217930739F3AF5FA43094
:1037C00081F7409391035093920310929303E0E0AA
:1037D000F0E020E03EE11AC0239FD0011124A35560
:1037E000B94F59968C915997882321F420939303CC
:1037F000FD0110C0873049F4309731F05A969C9102
:103800005A97828D891708F4FD012F5F243020F329
:1038100020939303309761F182E0818F80918D0333
:10382000848780918E03858780918F03868780911E
:103830009003878780E092E0938B828B958B848BBB
:1038400081E090E0918B808B138E81E0828F83E00A
:10385000808F168A80E1878B5483458377836683C4
:1038600088819981918380838A819B8193838283DC
:10387000CF01DF91CF910895BC018091AB0690916B
:10388000AC0608960E94471BE091AB06F091AC068F
:103890008091A20680878091A30681878091A406EB
:1038A00082878091A50683870895282F892F922FDC
:1038B0000895AC01FB0160939D07F0939E071616D7
:1038C000170664F42091A0063091A1068217930791
:1038D00029F0C901BA01AF010E94290108950F938F
:1038E0001F93CF93DF93C091AB06D091AC06843089
:1038F00009F4FEC12FE637E03093AA062093A9060B
:103900003093A1062093A006833059F4898D8F70DF
:10391000833009F055C788899989892B09F050C7E8
:1039200089C0823009F08AC0809190038F5F8093B4
:103930009003882399F480918F038F5F80938F0386
:10394000882361F480918E038F5F80938E03882398
:1039500029F480918D038F5F80938D0310929F06D1
:1039600010929E0610929E0710929D07298D273077
:1039700011F0253041F48A8D8F5F8A8F883709F0E6
:103980001FC7198E1DC7222309F41AC78889998970
:10399000892B09F44BC08A8D81508A8F8F5F09F083
:1039A0000FC73B8D383029F02150223048F4353094
:1039B00039F4198E80E88093A6060E94A111B7C53C
:1039C000353010F080E307C083E090E002C0880F3C
:1039D000991F3A95E2F78A8F8B8D8F5F8B8F898D38
:1039E00090E08F70907083309105D1F08430910514
:1039F00044F48130910509F482C3029709F0E0C6CE
:103A00000CC08630910509F425C58830910509F46C
:103A100021C5049709F0D4C61DC51092680772C36A
:103A200084E08093A6060E94A111B6C52F702330B2
:103A300009F0C6C688E08093A6066DC5853019F5E5
:103A4000E091A706F091A80684819581892B09F45D
:103A5000B7C61092AC061092AB06C9010C979093B2
:103A6000AA068093A9069093A1068093A0061092BF
:103A70009E0710929D0710929F0610929E0688E066
:103A80008093A60633C189010852104080914707F0
:103A9000853409F095C69091490780E020914A0746
:103AA000AC01420F511D80919E0690919F06841794
:103AB000950708F485C650939F0640939E06809113
:103AC0004D0790E08F739070892B09F079C6809133
:103AD0004E07882309F074C6409135075091360788
:103AE0008091DF019091E0014817590731F48091EE
:103AF000370790913807892B59F180915007813110
:103B000099F420915707309158078091E3019091E3
:103B1000E4012817390741F48091590790915A0719
:103B20008F5F9F4F09F45BC08091570790915807B2
:103B30008417950709F044C62091590730915A0718
:103B400080913707909138072817390709F038C650
:103B50000E941D168F5F9F4F09F032C6809150075B
:103B6000863009F42BC18131D1F1813009F028C6AA
:103B700080915B07883009F023C610925B07809123
:103B80005D0790915E072FEF873F920710F009962F
:103B900001C0089690935E0780935D07809153075C
:103BA0009091540790935807809357078091550739
:103BB0009091560790935A07809359078091350743
:103BC000909136079093540780935307809137075D
:103BD000909138079093560780935507F5C58091CB
:103BE0009E0690919F064C9790939F0680939E0609
:103BF00083E697E09093AA068093A90680916107D7
:103C000090916207892B31F00E9403168F5F9F4FBE
:103C100009F0D6C58FE997E09093A8068093A70690
:103C200046C02481358121153105E1F180915D0780
:103C300090915E0782179307A9F526813781211598
:103C4000310539F080915B0790915C0782179307EB
:103C500049F5208131818091DF019091E0012817A1
:103C6000390721F482819381892B59F18091E301F5
:103C70009091E4012817390729F4828193818F5F9D
:103C80009F4FF9F080915307909154078217930743
:103C900049F4209155073091560782819381281766
:103CA000390779F03B96F093A806E093A706E091D8
:103CB000A706F091A80687E0EB3CF80708F4B1CF1F
:103CC0007FC51092AC061092AB0682E08093A606E8
:103CD00083E697E09093AA068093A9069093A106A5
:103CE0008093A00610929E0710929D070E948C1848
:103CF00020919D0730919E072115310509F460C57B
:103D0000C9014C9690939F0680939E069093490715
:103D100080934A07E091A706F091A80680858093DA
:103D20004F0781E180935007C901089690935F0780
:103D300080936007109262071092610784819581D9
:103D400090935C0780935B078681978190935E07D1
:103D500080935D07809135079091360790935407C3
:103D600080935307809137079091380790935607B7
:103D700080935507808191819093580780935707CE
:103D80008281938190935A07809359078FE697E039
:103D90009093AA068093A9060E9403168095909599
:103DA0009093620780936107892B09F0E6C48FEF37
:103DB0009FEF9093620780936107DFC40E9407160C
:103DC0008F5F9F4F09F0FCC4CDEAD6E0898D882330
:103DD00029F120915D0730915E078C819D81281724
:103DE0003907E1F420915B0730915C078E819F8158
:103DF0002817390799F42091530730915407888187
:103E000099812817390751F42091550730915607A9
:103E10008A819B812817390709F48BC16E96F7E0D8
:103E2000C730DF0799F290F2809168078F73823074
:103E300011F580915D0790915E07909396038093B2
:103E400095031092930313C0E42FF0E0EE0FFF1FD1
:103E5000EB5DF84F2091950330919603808191811D
:103E60002817390709F471C04F5F409393034091BD
:103E70009303443048F38091680782FDA1C484E134
:103E8000F80181A388E290E090939F0680939E06BC
:103E900080E580A39091620780916607838F3091BF
:103EA000610780916507828F368F4091600780910E
:103EB0006407818F458F20915F0720939303809142
:103EC0006307808F248F9F5F978F992361F4832FDF
:103ED0008F5F868F882339F4842F8F5F858F8823A7
:103EE00011F42F5F248F20915B0730915C07309392
:103EF00096032093950380915D0790915E07F801EA
:103F0000958B848B378B268B809153079091540728
:103F100090935807809357078091550790915607C3
:103F200090935A07809359078091350790913607EF
:103F300090935407809353078091370790913807E7
:103F40009093560780935507FDC310929303C0E0EA
:103F5000D0E03EE136C0822F90E0FC0105E0EE0F9C
:103F6000FF1F0A95E1F7880F991FE81BF90BE3552E
:103F7000F94F818D882339F48EE1289FE0011124C7
:103F8000C355D94F22C08730C9F4209791F0822FB2
:103F900090E0FC01B5E0EE0FFF1FBA95E1F7880F46
:103FA000991FE81BF90BE355F94F928D8A8D8917FC
:103FB00028F4239FE0011124C355D94F2F5F20938C
:103FC000930320919303243030F2209709F4F8C32F
:103FD000D093AC06C093AB0683E08A8F888F1E8A8D
:103FE00084E08F8B1B8E80915D0790915E079D838F
:103FF0008C8380915B0790915C079F838E83809177
:104000005307909154079983888380915507909125
:1040100056079B838A8381E0898F80918D038C87EB
:1040200080918E038D8780918F038E87809190037E
:104030008F8781E090E0998B888B809162078B87D6
:10404000809161078A8780916007898780915F07E7
:10405000888781E090E00E943C1C8091670790E097
:10406000807F9070813591050CF449C010929303C4
:1040700034C0F901E75CF84F86A980939403882344
:10408000F1F1813021F44F5F4093930326C08230D9
:10409000C1F487A98430A9F430AD20E081AD90E06F
:1040A000822B932B9093960380939503F2E08130BB
:1040B0009F0710F080E092E09B8B8A8B9D8B8C8B0E
:1040C0001EC090919303E92FF0E0E75CF84F87A9B9
:1040D0008823A9F0890F8093930340919303242FA1
:1040E00030E08091670782958F7090E00597880F88
:1040F000991F880F991F281739070CF4BACF80E150
:10410000809368078091680782608093680792E0D7
:1041100090936F0784E080937007909371071092DB
:1041200072078CE290E090939F0680939E0680E653
:10413000B7C2D093AC06C093AB061092A60680918E
:104140006807482F50E082FF03C0198E80E251C2F9
:104150008091670782958F70880F880F80939303F3
:1041600020919E0630919F0624513040281B310932
:1041700030939F0620939E06898D8F70823029F49C
:104180004F7350704231510509F1232B39F480915E
:10419000680790E083709070892BC1F090915F0761
:1041A0008885981709F072C29091600789859817E1
:1041B00009F06CC2909161078A85981709F066C270
:1041C000909162078B85981709F060C2809168070B
:1041D00084FF51C0688979896115710509F44BC064
:1041E000CE010C960E94471B209163078091A20686
:1041F000281709F040C0909164078091A306981792
:10420000D1F5909165078091A4069817A1F590913A
:1042100066078091A506981771F52C878091A306F3
:104220008D878091A4068E878091A5068F878B8DC0
:104230008823D1F42E89988D8A8D981B822F86959C
:1042400086958695981B392F320F3E8B8F89282FA4
:1042500026952695821B97FD9195890F8F8B369514
:1042600036953695830F888F81E08093A606888DDA
:104270008A8F198A188A898D282F30E0C9018F709A
:1042800090708430910509F4B9C1853091055CF4D2
:104290008230910591F1833091050CF0B1C0019706
:1042A00009F08EC210C08630910509F4E7C186304E
:1042B00091050CF4C3C18730910509F4E7C1089753
:1042C00009F07EC290C18091A60680FF79C283E08A
:1042D000898F80E48093A606198A188A20919E0609
:1042E00030919F062115310509F411C182E48093B4
:1042F000A606C9010E943C1C0AC18091A60680FF47
:1043000074C0809168078F73823109F06EC080910C
:10431000670790E0807F9070813591050CF449C06B
:104320001092930334C0F901E75CF84F86A980939B
:1043300094038823F1F1813021F44F5F409393037C
:1043400026C08230C1F487A98430A9F430AD20E0C2
:1043500081AD90E0822B932B9093960380939503ED
:1043600022E08130920710F080E092E09B8B8A8BF4
:104370009D8B8C8B1EC090919303E92FF0E0E75C3E
:10438000F84F87A98823A9F0890F80939303409160
:104390009303242F30E08091670782958F7090E01F
:1043A0000597880F991F880F991F281739070CF454
:1043B000BACF83E0898F80915F07888780916007FB
:1043C0008987809161078A87809162078B8781E066
:1043D00090E00E943C1C82E48093A606198A188A09
:1043E00010929F0610929E0692C080E28093A606CD
:1043F0000E94A111E091AB06F091AC06118E3BCD6D
:104400008091680780FF2AC024FD28C08889998987
:10441000892B09F0D5C180919E0690919F06019647
:104420000E943C1C2091A606822F80618093A606E4
:1044300080919E0690919F06892B19F0226120930E
:10444000A6060E94A11181E090E0998B888B88E0FC
:10445000898F1B8E81E1809368071BC185FF21C076
:1044600060916D07362F20E040916E0750E0242BBD
:10447000352B8091A9069091AA06820F931F9093E5
:10448000AA068093A906962F80E0842B952B209175
:104490009E0630919F06281B390B30939F06209370
:1044A0009E0620919E0630919F062115310559F0F8
:1044B000898D84FD08C08091A60682608093A6063F
:1044C000C9010E943C1C9091690780E020916A0715
:1044D000820F911D90939603809395032C893D89BB
:1044E0002817390710F0892B21F430939603209375
:1044F000950380919503909196039B8B8A8B809175
:10450000A60690E083709070892B09F459C110922F
:104510009E0710929D070E94A1118091A606282F48
:1045200085FF07C010929E0710929D07198E84E1A7
:1045300092CF84FF0AC010929E0710929D0781E0DF
:1045400090E0998B888B84E083CF80919D07909138
:104550009E07892B01F120FF02C0198A188A8889D9
:1045600099890097A1F42A893B8980919D079091B0
:104570009E072817390720F430939E0720939D0744
:1045800080919D0790919E07998B888B04C0909392
:104590009E0780939D071B8E8091A0069091A10697
:1045A0009093AA068093A90680919D0790919E07FB
:1045B000892B59F088899989009739F088969093CA
:1045C0009F0680939E0688E10BC08091A60681FF1E
:1045D000F7C088E290E090939F0680939E0680E16A
:1045E000809368075CC08091A60680FFE9C0198EA1
:1045F00080E18093A6060E94A111E2C080919E06F0
:1046000090919F06009711F00E943C1C80916807D2
:104610009091A60680FF0BC090FF06C087E0898FAF
:104620001A8E198A188A19C086E0898F16C090FFE1
:104630001EC085E0898F198A188AC2C080919E06A3
:1046400090919F06009711F00E943C1C8091680792
:1046500080FF0DC087E0898F1A8E81E090E00E9474
:104660003C1C80E18093A6060E94A1110FC080919E
:104670009E0690919F06892B49F4A2C08091A606C0
:1046800080FF9EC087E0898F1A8E9AC080E1F80172
:1046900081A388E290E090939F0680939E0680E538
:1046A0008093670788858093630789858093640773
:1046B0008A85809365078B85809366078C858093B8
:1046C0005F078D85809360078E85809361078F8556
:1046D0008093620786E0809350078C819D81909340
:1046E0005C0780935B078E819F8190935E07809328
:1046F0005D0780913507909136079093540780931A
:10470000530780913707909138079093560780930D
:1047100055078881998190935807809357078A811C
:104720009B8190935A0780935907898D84FF05C018
:1047300010926A071092690705C082E080936907AA
:1047400010926A0780E480934F0780919F068093C0
:10475000490780919E0680934A0710926E07109237
:104760006D0710926C0710926B070E9407168095D8
:10477000909590936C0780936B0785E4809347072F
:104780001092480710924E0710924D0780918B03AC
:1047900090918C03019690938C0380938B0390935C
:1047A0004B0780934C0710925207109251070E94BA
:1047B0001D1680959095909352078093510704C0E1
:1047C00010929F0610929E061092A606DF91CF913E
:1047D0001F910F9108950F931F93CF93DF93EC01D7
:1047E0008B0120919103309192036BE070E02F5F79
:1047F0003F4F8DE72030380710F020E030E1522F96
:10480000432FA0E011C08A2F90E0869FF001879F80
:10481000F00D969FF00D1124E156F84F848195819B
:10482000AF5F8417950719F3A43069F720939103BC
:10483000309392031092930340E0ABE0B0E01CC0D1
:10484000542F5F5F842F90E08A9FF0018B9FF00DC3
:104850009A9FF00D1124E156F84F84819581892BA0
:1048600051F4409393038BE0489FF0011124E156EB
:10487000F84F49F41DC0452F443010F34093930383
:10488000E0E0F0E015C0348325831783068320978A
:1048900029F4108211821282138208C088819981C2
:1048A000918380838A819B819383828380E4808744
:1048B000CF01DF91CF911F910F910895DF92EF9279
:1048C000FF920F931F93CF93DF93DC01062FD72E18
:1048D0001092F30360E01BE02BC0619FF0011124F4
:1048E000E956FC4F408151814115510501F122816A
:1048F000338121153105D9F08D919C911197841741
:104900009507A9F412968D919C911397821793079E
:1049100071F46093F303EF012496802F9D2D9C0189
:10492000D90186E00D9009928150E1F767C06F5F71
:10493000683098F21092F30320E03BE011C0239F0F
:10494000F0011124E956FC4F80819181892B39F4C3
:1049500082819381892B19F42093F3033CC02F5F4C
:10496000283068F32093F3032830A9F51092F6035A
:104970001092F4031091F503C12FD0E060E070E0D5
:1049800040E08BE0E82EF12C18C0842F90E08E9D43
:10499000F0018F9DF00D9E9DF00D1124E956FC4F06
:1049A00052859E01251B3109872F90E082179307BE
:1049B0001CF4712F751B642F4F5F483030F36093E8
:1049C000F4037093F6036093F3038BE0689FF001A8
:1049D0001124E956FC4F8D919D910D90BC91A02D15
:1049E000EF0189939993A993B993202F3D2DC90184
:1049F000DC0186E00D9009928150E1F78091F5038A
:104A00008287DF91CF911F910F91FF90EF90DF9000
:104A1000089580919E0690919F060E9790939F0611
:104A200080939E0680913507909136072091530719
:104A30003091540782279327209131073091320714
:104A400082239323892BC1F48091370790913807F3
:104A500020915507309156078227932720913307DD
:104A60003091340782239323892B31F483E597E037
:104A70006FE377E00E945E240895CF93DF938091E7
:104A80009E0690919F068A9728F410929F06109296
:104A90009E06A6C010929F0610929E06C9E3D7E01C
:104AA00080914D0790914E0721E08030920729F0C8
:104AB0008050924009F094C076C020915F073091F9
:104AC000600780913507909136072817390709F05C
:104AD00087C02091610730916207809137079091DC
:104AE00038072817390709F07BC0CE014C96BE0164
:104AF0006A5E7F4F0E945E2480E092E090934E07B2
:104B000080934D07DE019096FE01769686E0019037
:104B10000D928150E1F7AFE4B7E0E5E8F3E086E01D
:104B200001900D928150E1F7AFE3B7E0E5E8F3E0E3
:104B300086E001900D928150E1F7E9E3F7E0DF01B3
:104B4000909686E00D9001928150E1F78091550793
:104B5000909156079093600780935F078091570765
:104B60009091580790936207809361078091350771
:104B70009091360790935607809355078091370799
:104B800090913807909358078093570788E096E0F4
:104B900090934607809345078AE290E090939F06A2
:104BA00080939E061DC020915F0730916007809121
:104BB0003507909136072817390791F4209161073E
:104BC000309162078091370790913807281739078D
:104BD00039F4CE014C96BE016A5E7F4F0E945E247E
:104BE000DF91CF91089540915707509158078091D8
:104BF000E7019091E8014817590789F48091590716
:104C000090915A078F5F9F4F51F4A9E3B7E0EBEE05
:104C1000F1E086E001900D928150E1F7CDC08091E6
:104C200035079091360784279527209131073091D9
:104C3000320782239323892B91F460915907709155
:104C40005A07809137079091380786279727209138
:104C500033073091340782239323892B89F0809185
:104C60002D0790912E079093F0038093EF0380918E
:104C70002F07909130079093F2038093F10308C0BF
:104C80005093F0034093EF037093F2036093F103AA
:104C90001092F3036091EF037091F0034091F103E0
:104CA0005091F20320E03BE013C0239FF001112458
:104CB000E956FC4F808191816817790741F4828120
:104CC00093814817590719F42093F3036DC02F5FA0
:104CD000283058F32093F303283009F065C089E3A6
:104CE00097E06FEF70E046E050E00E943201E9E5A6
:104CF000F7E086E0DF011D928A95E9F77A97A5E84B
:104D0000B3E086E00D9001928150E1F7AFE4B7E0A7
:104D1000E5E8F3E086E001900D928150E1F78091A3
:104D2000EF039091F0039093600780935F07809169
:104D3000F1039091F2039093620780936107809151
:104D400035079091360790935607809355078091C9
:104D5000370790913807909358078093570780E062
:104D600091E090934E0780934D079093480780936E
:104D7000470788E090E090934A078093490786E0D0
:104D800080934B0784E080934C0788E096E09093F3
:104D90004607809345078FE697E09093AA06809395
:104DA000A9068AE290E01CC0A9E3B7E0349686E049
:104DB00001900D928150E1F7AFE3B7E0E5E8F3E051
:104DC00086E001900D928150E1F788E090E09093A9
:104DD00046078093450780919E0690919F060E9608
:104DE00090939F0680939E0608951092F3039BE094
:104DF0000CC0899FF0011124E956FC4F10821182EA
:104E0000128213828F5F8093F3038091F3038830C3
:104E100080F30895882319F420E030E013C08F3F19
:104E200029F42091FB033091FC030CC090E0FC01BD
:104E3000EE0FFF1FEE0FFF1FE80FF91FE250FC4FB0
:104E400022813381C90108950F931F93CF93DF937C
:104E50008C01EB018AE060E00E94F6338AE78EBDA8
:104E60000DB407FEFDCF08C088818EBD0DB407FECE
:104E7000FDCF01501040219601151105A9F78AE0D8
:104E800061E00E94F633DF91CF911F910F91089559
:104E90000F931F93CF93DF93EC018B018AE060E0C7
:104EA0000E94F6338AE38EBD0DB407FEFDCF09C024
:104EB0001EBC0DB407FEFDCF21978EB5F80181937E
:104EC0008F012097A9F78AE061E00E94F633DF9115
:104ED000CF911F910F910895FF920F931F93082F69
:104EE000162FF42E8AE060E00E94F6331F71102B1B
:104EF0001EBD0DB407FEFDCFFEBC0DB407FEFDCFF9
:104F00008AE061E00E94F6331F910F91FF900895AF
:104F10001F93CF93DF93182FC82FD0E0C076D070A7
:104F20008091980190E0C817D90791F080EA6FE16D
:104F300043E00E946C2735E0D595C7953A95E1F797
:104F400080E86FE14C2F0E946C2710761093980137
:104F5000DF91CF911F910895FF920F931F93182F08
:104F6000062FF72E0E94882780E4612F402F0E9491
:104F70006C271F5F80E4612F4F2D0E946C271F91CB
:104F80000F91FF900895CF92DF92EF92FF920F93CF
:104F90001F93CF93DF937B01EA01D22EC32E90E0C3
:104FA0008C01000F111F000F111F080F191F025055
:104FB0001C4FF801608171816E0D7F1D82E00E949F
:104FC000AC27F801428153814E195F092D2D3C2DEC
:104FD000C9016C014817590708F46A01C601BE01EE
:104FE0000E942427C601DF91CF911F910F91FF905E
:104FF000EF90DF90CF900895EF92FF920F931F9361
:10500000CF93DF93982F8B01F42EE52E8F3F41F144
:1050100085E0989FE0011124C250DC4F07C06F5F0C
:105020007740C9EFD3E006C0C9EFD3E0688179814A
:10503000600F711F80E00E94AC274A815B81401B9A
:10504000510B8F2D9E2D9C014217530708F49A0196
:10505000C901DF91CF911F910F91FF90EF900895BB
:105060006091F9037091FA03600F711F88E060305E
:105070007807D0F2D4CFEF92FF920F931F937A016B
:10508000A9010E94FC27182F092FB7010E94482769
:10509000812F902F1F910F91FF90EF9008956091B5
:1050A000F7037091F8036115710519F46FEF77E05C
:1050B00002C0615070408CE00E94AC2708950E94AD
:1050C0004F2808950F931F93182F062F0E948827AB
:1050D00080E4612F402F0E946C271F910F9108954B
:1050E0000F931F93CF93DF93EC01862FBA01A90191
:1050F0000E94FC278C01015010408AE060E00E9471
:10510000F6338AE38EBD0DB407FEFDCF40E050E0DC
:1051100017C01EBC0DB407FEFDCF9EB51EBC0DB45E
:1051200007FEFDCF8EB5392F20E0B901680F711D44
:10513000C60FD71FC617D70708F421964E5F5F4FDB
:105140004017510730F34017510769F41EBC0DB4E6
:1051500007FEFDCF2EB5922F80E0C80FD91FC817CC
:10516000D90708F421968AE061E00E94F633CE0167
:10517000DF91CF911F910F9108950F931F93182FD7
:10518000062F8AE060E00E94F633802F8F71812B1A
:105190008EBD0DB407FEFDCF1EBC0DB407FEFDCFC6
:1051A00007FF04C01EBC0DB407FEFDCF8AE061E01E
:1051B0000E94F6338EB51F910F9108951F93182FFB
:1051C0000E94882780E0612F0E94BD281F910895CA
:1051D000FF920F931F93CF93DF9389E30E94DE2802
:1051E000882309F450C06091F7037091F803EB0134
:1051F000269688E0C030D80718F0EB01C95FD74089
:1052000080E00E94AC278AE360E00E94BD28082F5E
:1052100010E01093F8030093F7038AE360E00E9424
:10522000BD28382F20E0202B312B3093F80320931A
:10523000F7038AE360E00E94BD28F82E8AE360E06D
:105240000E94BD28082F8AE360E00E94BD28182F25
:1052500080E86EE140E40E946C2717FF11C0D093F4
:10526000FA03C093F9032F2D30E0902F80E0822BBA
:10527000932B04979093FC038093FB038FEF03C061
:105280000E944F2880E0DF91CF911F910F91FF90F6
:1052900008951F939C01162F82E0B9010E94AC274C
:1052A0008AE060E00E94F6338AE78EBD0DB407FE07
:1052B000FDCF1EBD0DB407FEFDCF8AE061E00E9468
:1052C000F6331F910895BC0180E00E94AC278AE06C
:1052D00060E00E94F6338AE38EBD0DB407FEFDCF79
:1052E0001EBC0DB407FEFDCF8AE061E00E94F633DC
:1052F0008EB50895EF92FF920F931F93CF93DF9394
:105300007C01EB014130510541F4CB010E9463293E
:10531000682FC7010E9449292AC021978E01040FD6
:10532000151F219680E1BE010E94AC2784E1B701E0
:105330000E94AC27C050D84030F488E000301807F5
:1053400010F00F5F174082E1B8010E94AC2780EA9D
:105350006FE140E10E946C2780E86FE140E20E942B
:105360006C2780E06FE10E94BD2885FDFACFDF91B8
:10537000CF911F910F91FF90EF9008950F931F937E
:10538000982FDB014F3F39F185E0489FF001112450
:10539000E250FC4F05C06F5F774006C0E9EFF3E0D5
:1053A00060817181620F731F892F90E0FC01EE0F05
:1053B000FF1FEE0FFF1FE80FF91FE250FC4F808127
:1053C00091818A0F9B1FA8010E947A290E944F2871
:1053D0001F910F9108956091F9037091FA03620F84
:1053E000731F88E060307807C8F2D5CFFF920F9323
:1053F0001F93CF93DF9390E0FC01EE0FFF1FEE0FA2
:10540000FF1FE80FF91FE250FC4FC081D1812197A7
:1054100002811381CE010E946329F82E882321F096
:10542000CE0160E00E94492984E0BE010E94AC27C1
:105430000C0F1D1F86E0B8010E94AC2780E86FE1C9
:1054400048E00E946C278CE10E94DE2881FF05C0A5
:1054500080EA6FE148E00E946C27FF2021F0CE0136
:105460006F2D0E944929DF91CF911F910F91FF90DD
:1054700008950F931F93982F8B0184ED692F0E943D
:10548000622886EDB8010E94AC2704C08FE090E04E
:105490000E9472338AEE0E94DE2880FDF7CF1F91B2
:1054A0000F9108950F931F938C010E94FF2B8AE0A8
:1054B00061E00E94B7338AE061E00E94F6338BE03E
:1054C00061E00E94B7338DE061E00E94B7338CE069
:1054D00060E00E94B7338AE061E00E94B7338BE05E
:1054E00060E00E94F6338DE060E00E94F63380E5D4
:1054F0008CBD8DB581608DBD8FEF60E04FEF0E9458
:105500006C2762E370E080E090E00E941933109213
:10551000F8031092F70388E060E070E00E94AC2787
:105520008CE060E070E00E94AC278AE06FEF77E0EB
:105530000E94AC2788E361EB0E94622888E26FE357
:1055400070E30E94AC2780E369EF77EF0E94AC27FD
:1055500080EC6DE070E00E94AC2780E862EC42E3F2
:105560000E946C2786EC62E17CE00E94AC2784EC10
:1055700062E10E9462288AEC6CED75E00E94AC2723
:1055800084EEF80160810E94622885EEF801618155
:105590000E94622882EEF80162810E94622883EEF6
:1055A000F80163810E94622880EEF80164810E9404
:1055B000622881EEF80165810E94622880E160E046
:1055C00071E00E94392A8FE10E94882780E86BE110
:1055D00040EC0E946C2780E86FE144E00E946C2759
:1055E00084E166E774E00E94392A1F910F910895C3
:1055F000882309F1AEEFB3E095E014962C9114974F
:10560000281789F490E0FC01EE0FFF1FEE0FFF1F3B
:10561000E80FF91FE250FC4F848114968C9313829B
:10562000128214820895222331F0299FD00111247F
:10563000A250BC4FE2CF089590E0FC01EE0FFF1F97
:10564000EE0FFF1FE80FF91FE250FC4F80819181A0
:10565000860F971F9183808382819381861B970B8E
:1056600093838283089590E0FC01EE0FFF1FEE0FFD
:10567000FF1FE80FF91FE250FC4F80819181860FD8
:10568000971F91838083538342830895CF92DF9243
:10569000EF92FF920F931F93CF93DF936C012091B2
:1056A000FE033091FF032150384EC0E0D0E050E0BF
:1056B000AEEFB3E060E078E115E014964C911497FA
:1056C000442311F4F9010EC0842F90E0FC01EE0F89
:1056D000FF1FEE0FFF1FE80FF91FE250FC4F019074
:1056E000F081E02D8D919C911197E81BF90B12969A
:1056F0008D919C911397E81BF90BEC15FD0539F47E
:1057000085E0589FE0011124C250DC4F53C0CE16F3
:10571000DF0648F4E617F70730F4519FE001112443
:10572000C250DC4FBF01442331F4209709F042C03E
:10573000EEEFF3E02AC0419FD0011124A250BC4FEC
:10574000542FBBCF7A01E20EF31E082F10E0E801C0
:10575000CC0FDD1FCC0FDD1FC00FD11FC250DC4F9F
:1057600068817981E616F70639F04A815B81C701C5
:105770000E947A29F982E882F801EE0FFF1FEE0FEE
:10578000FF1FE00FF11FE250FC4F848142815381E3
:10579000208131818823B1F68091FE039091FF032F
:1057A000821B930B841B950B8150984E8C159D0585
:1057B000D8F0EF0141E0E3E0F4E082819381892BAE
:1057C00029F04F5F453381F03596F7CF8A819B8171
:1057D00028813981820F931F91838083D382C28273
:1057E0008C8184834C8301C040E0842FDF91CF9172
:1057F0001F910F91FF90EF90DF90CF90089589E077
:1058000091E0EEEFF3E0DF019C011D92215030406A
:10581000E1F781E098E09093FF038093FE031092FC
:10582000010410920004109202040895FC012FEF6D
:105830003FEF338322838AE090E09783868381E081
:1058400080878EE591E095838483318320838CE388
:1058500090E090939A01809399011092070510921D
:1058600008051092090510920A05089520E080911C
:10587000070590910805A0910905B0910A050097C8
:10588000A105B10509F021E0822F089510920705C6
:10589000109208051092090510920A05089560916A
:1058A0000705709108058091090590910A050895F2
:1058B0002F923F924F925F926F927F928F929F9220
:1058C000AF92BF92CF92DF92EF92FF920F931F930E
:1058D000DF93CF93CDB7DEB762970FB6F894DEBFF4
:1058E0000FBECDBF3C0180911105909112056FE173
:1058F00070E00E9494394B017B0100E010E02091A0
:10590000990130919A01442737FD4095542FC801E1
:10591000B7010E9475390E9484382AE037ED43E2CE
:105920005CE30E9412390E945838A8019701220FA7
:10593000331F441F551F2E0D3F1D401F511F59017E
:105940006A01A61AB70AC80AD90AAD82BE82CF82F6
:10595000D8865B016C01A20EB31EC41ED51EA9829F
:10596000BA82CB82DC82AA24BB24650121E030E02C
:105970003A87298717012801261A370A480A590A3F
:10598000A8019701260F371F481F591F2F87388BF3
:10599000498B5A8B7AC0E985FA85EE0FFF1FEF5EBF
:1059A000FA4F808191819C0140E050E0221633063D
:1059B0004406550658F58F859889A989BA8928170C
:1059C00039074A075B0710F5E985FA85EE0FFF1FD7
:1059D000ED5EFA4F0190F081E02D7F0100E010E0D4
:1059E000EB86FC860D871E878D819E81AF81B885F1
:1059F0008E159F05A007B10748F489819A81AB8174
:105A0000BC81E816F9060A071B0778F1ED80FE80D5
:105A10000F811885E216F3060407150758F58981EA
:105A20009A81AB81BC81281739074A075B0710F5BB
:105A3000E985FA85EE0FFF1FED5EFA4F80819181B7
:105A4000A0E0B0E0281639064A065B0698F4EF8419
:105A5000F88809891A898E159F05A007B10750F4A7
:105A60000894A11CB11CC11CD11CAA0CBB1CCC1CD1
:105A7000DD1C05C07A866986AA24BB2465010985D8
:105A80001A850E5F1F4F1A87098729853A852615C3
:105A9000370508F480CFA6019501569547953795AF
:105AA000279587E068167104C0F0209307053093AE
:105AB00008054093090550930A05769467947092FF
:105AC0000C0560920B0590920E0580920D0581E009
:105AD00090E09093100580930F0580E0211531052B
:105AE0004105510509F081E062960FB6F894DEBFDA
:105AF0000FBECDBFCF91DF911F910F91FF90EF901F
:105B0000DF90CF90BF90AF909F908F907F906F90DD
:105B10005F904F903F902F9008952F923F924F9219
:105B20005F926F927F928F929F92AF92BF92CF922D
:105B3000DF92EF92FF920F931F93DF93CF93CDB736
:105B4000DEB762970FB6F894DEBF0FBECDBF3C0143
:105B500080911105909112056AE070E00E949439DD
:105B60004B017B0100E010E02091990130919A01F6
:105B7000442737FD4095542FC801B7010E9475395D
:105B80000E9484382AE037ED43E25CE30E94123938
:105B90000E945838A8019701220F331F441F551F38
:105BA00059016A01A61AB70AC80AD90AAD82BE828B
:105BB000CF82D8865B016C01A20EB31EC41ED51E17
:105BC000A982BA82CB82DC82AA24BB24650121E0AF
:105BD00030E03A87298717012801261A370A480A30
:105BE000590AA8019701260F371F481F591F2F87F1
:105BF000388B498B5A8B7AC0E985FA85EE0FFF1FE7
:105C0000EF5EFA4F808191819C0140E050E02216C6
:105C100033064406550658F58F859889A989BA89AF
:105C2000281739074A075B0710F5E985FA85EE0F53
:105C3000FF1FED5EFA4F0190F081E02D7F0100E043
:105C400010E0EB86FC860D871E878D819E81AF81DB
:105C5000B8858E159F05A007B10748F489819A8100
:105C6000AB81BC81E816F9060A071B0778F1ED80C5
:105C7000FE800F811885E216F3060407150758F514
:105C800089819A81AB81BC81281739074A075B0754
:105C900010F5E985FA85EE0FFF1FED5EFA4F808162
:105CA0009181A0E0B0E0281639064A065B0698F418
:105CB000EF84F88809891A898E159F05A007B10716
:105CC00050F40894A11CB11CC11CD11CAA0CBB1C13
:105CD000CC1CDD1C05C07A866986AA24BB2465011C
:105CE00009851A850E5F1F4F1A87098729853A850E
:105CF0002615370508F480CFA601950156954795DE
:105D00003795279587E068167104C0F02093070542
:105D1000309308054093090550930A0576946794DB
:105D200070920C0560920B0590920E0580920D0505
:105D300082E090E09093100580930F0580E021159C
:105D400031054105510509F081E062960FB6F894DE
:105D5000DEBF0FBECDBFCF91DF911F910F91FF909E
:105D6000EF90DF90CF90BF90AF909F908F907F90FB
:105D70006F905F904F903F902F9008952F923F9299
:105D80004F925F926F927F928F929F92AF92BF924B
:105D9000CF92DF92EF92FF920F931F93DF93CF93F7
:105DA000CDB7DEB76C970FB6F894DEBF0FBECDBF90
:105DB0004C01809111059091120567E470E00E94FA
:105DC00094391B015B01CC24DD2420919901309191
:105DD0009A01442737FD4095542FC601B5010E9412
:105DE00075390E9484382AE037ED43E25CE30E9473
:105DF00012390E9458387B018C01D601C50142E05E
:105E0000880F991FAA1FBB1F4A95D1F79C01AD01AE
:105E10002E193F09400B510B2D8B3E8B4F8B588F0A
:105E2000A8019701280F391F4A1F5B1F298B3A8B46
:105E30004B8B5C8BC601B5012BE030E040E050E0BD
:105E40000E9475399B01AC012E193F09400B510B83
:105E50002D873E874F87588BA8019701260F371F44
:105E6000481F591F29873A874B875C87D601C50190
:105E700033E0880F991FAA1FBB1F3A95D1F78A0DEF
:105E80009B1DAC1DBD1D9C01AD012E193F09400B92
:105E9000510B2D833E834F835887A8019701280F0C
:105EA000391F4A1F5B1F29833A834B835C83C601DA
:105EB000B50126E030E040E050E00E9475392B014A
:105EC0003C014E185F08600A710A57016801A60E6E
:105ED000B71EC81ED91EA98EBA8ECB8EDC8EEE24BC
:105EE000FF24870161E070E070C0FB01EE0FFF1F2F
:105EF000EF5EFA4F808191819C0140E050E08D89F6
:105F00009E89AF89B88D82179307A407B50720F53E
:105F1000A988BA88CB88DC882A153B054C055D0525
:105F2000D8F4FB01EE0FFF1FED5EFA4F80819181E7
:105F3000A0E0B0E0AD84BE84CF84D888A816B906AE
:105F4000CA06DB0648F4A984BA84CB84DC848A15AB
:105F50009B05AC05BD0570F18D819E81AF81B88533
:105F600082179307A407B50750F5A980BA80CB80A4
:105F7000DC802A153B054C055D0508F5FB01EE0F9D
:105F8000FF1FED5EFA4F80819181A0E0B0E04816DE
:105F900059066A067B0698F4298D3A8D4B8D5C8DE7
:105FA00082179307A407B50750F40894E11CF11C6D
:105FB000011D111DEE0CFF1C001F111F04C0B401B8
:105FC000EE24FF2487016E5F7F4F6815790508F482
:105FD0008CCFA8019701569547953795279587E06F
:105FE00088169104C0F0209307053093080540936C
:105FF000090550930A059694879490920C05809217
:106000000B0530920E0520920D0583E090E09093F1
:10601000100580930F0580E02115310541055105DC
:1060200009F081E06C960FB6F894DEBF0FBECDBFCD
:10603000CF91DF911F910F91FF90EF90DF90CF9064
:10604000BF90AF909F908F907F906F905F904F9098
:106050003F902F900895CF93DF93EA01E7EBF5E0AF
:1060600040E050E00CC060FD02C0322F01C031E3BF
:1060700031934F5F5F4F969587957795679561153B
:1060800071058105910579F7BE01641B750BDE0171
:10609000AA54BA4FE7E9F5E040E050E00BC04617DC
:1060A000570718F08C91808301C020834F5F5F4FAA
:1060B000119731964C175D0790F3C956DA4F188245
:1060C00087E995E0DF91CF91089520E30E942B307E
:1060D0000895CF92DF92EF92FF920F931F93CF9389
:1060E000DF930E94F3326B017C018091D90590917E
:1060F000DA058601081B190B1093E0050093DF05F4
:1061000083E109381807C0F120911105309112057B
:10611000C901885C90408017910750F528533F4F84
:106120000217130728F58091D7059091D80501969D
:106130009093D8058093D705C091DD05D091DE05F9
:106140002197D093DE05C093DD05029789F4CE0137
:106150000E94582C882341F4CE010E948D2D882363
:1061600019F4CE010E94BE2E1092D8051092D705C8
:106170001092DE051092DD058091DD059091DE051F
:106180008334910540F01092DE051092DD051092E7
:10619000D8051092D7058091DD059091DE05FC01B0
:1061A000EE0FFF1FEF5EFA4F11830083019690936D
:1061B000DE058093DD05C092D905D092DA05E09224
:1061C000DB05F092DC05DF91CF911F910F91FF90DD
:1061D000EF90DF90CF9008950F931F938C01FC01F7
:1061E00080810E9430328FEF9FEFF801918380838E
:1061F0001F910F910895FC01808191812FEF8F3FB6
:10620000920791F010920705109208051092090567
:1062100010920A0510920C0510920B0569E670E3C6
:1062200041E050E00E940D320895FC0171836083CB
:106230000E94FB300895AF92BF92DF92EF92FF92DF
:106240000F931F93CF93DF93EC017B015A010881D9
:1062500019818A819B818F5F9F4F91F13FEF0F3FA3
:10626000130711F4DD2405C0CE010E94EC30DD24BB
:10627000D3948A8161E00E94F6338C819D819C01D8
:10628000E29EC001E39E900DF29E900D11240E94AB
:1062900072338A8160E00E94F6338C819D819C017B
:1062A000A29EC001A39E900DB29E900D11240E944B
:1062B0007233DD2029F019830883CE010E94FB3060
:1062C000DF91CF911F910F91FF90EF90DF90BF90E2
:1062D000AF900895FC018085813031F4CF0161E0F9
:1062E00070E04FE150E007C0823041F4CF0161E03F
:1062F00070E04AE050E00E941B310895833039F489
:10630000CF0161E070E047E450E00E941B31089546
:10631000FC018085813021F4CF0163E070E005C08D
:10632000823041F4CF0162E070E041E050E00E9431
:106330001B310895833039F4CF0169E070E046E005
:1063400050E00E941B310895FC018085813031F4BA
:10635000CF0161E070E043E050E007C0823041F4DB
:10636000CF0161E070E042E050E00E941B310895EF
:10637000833039F4CF0164E070E04BE050E00E94DC
:106380001B310895CF92DF92EF92FF920F931F93EC
:10639000CF93DF938C016B01EE24FF2416C0803372
:1063A00019F0813341F404C0C8010E94A43103C034
:1063B000C8010E94883121968881882381F7C8010D
:1063C0000E946A310894E11CF11CF80186819781D2
:1063D000E816F90614F4E601EFCFDF91CF911F9193
:1063E0000F91FF90EF90DF90CF9008950F931F9340
:1063F0008C01CB01BA01A9010E946530BC01C80122
:106400000E94C2311F910F910895FC01862F628373
:10641000738361E00E94B7330895823000F5E82F5E
:10642000F0E0EE0FFF1FEF51FA4F71836083882376
:1064300019F08130A1F408C0809169008C7F842B11
:1064400080936900E89A089580916900440F551F70
:10645000440F551F837F842B80936900E99A089528
:10646000823080F4882319F0813021F402C0E8984A
:1064700001C0E998E82FF0E0EE0FFF1FEF51FA4F4F
:106480001182108208951F920F920FB60F9211245D
:106490002F933F934F935F936F937F938F939F932C
:1064A000AF93BF93EF93FF938091E1059091E20545
:1064B000892B29F0E091E105F091E2050995FF9122
:1064C000EF91BF91AF919F918F917F916F915F916C
:1064D0004F913F912F910F900FBE0F901F901895E5
:1064E0001F920F920FB60F9211242F933F934F9349
:1064F0005F936F937F938F939F93AF93BF93EF932C
:10650000FF938091E3059091E405892B29F0E091B8
:10651000E305F091E4050995FF91EF91BF91AF91EB
:106520009F918F917F916F915F914F913F912F91AB
:106530000F900FBE0F901F9018951F920F920FB6DD
:106540000F9211242F933F938F939F93AF93BF93F9
:106550008091E9059091EA05A091EB05B091EC05D9
:106560003091ED050196A11DB11D232F2D5F2D3713
:1065700020F02D570196A11DB11D2093ED058093AC
:10658000E9059093EA05A093EB05B093EC058091A3
:10659000E5059091E605A091E705B091E805019623
:1065A000A11DB11D8093E5059093E605A093E70535
:1065B000B093E805BF91AF919F918F913F912F913B
:1065C0000F900FBE0F901F9018958FB7F8942091E1
:1065D000E9053091EA054091EB055091EC058FBF3C
:1065E000B901CA0108959FB7F8942091E50530914B
:1065F000E6054091E7055091E80586B5A89B06C0E1
:106600008F3F21F02F5F3F4F4F4F5F4F9FBF542F62
:10661000432F322F2227280F311D411D511D82E0AB
:10662000220F331F441F551F8A95D1F7B901CA01A4
:1066300008959B01AC017FB7F8948091E505909196
:10664000E605A091E705B091E80566B5A89B05C0F1
:106650006F3F19F00196A11DB11D7FBFBA2FA92F61
:10666000982F8827860F911DA11DB11D62E0880F0C
:10667000991FAA1FBB1F6A95D1F7BC012DC0FFB798
:10668000F8948091E5059091E605A091E705B09119
:10669000E805E6B5A89B05C0EF3F19F00196A11DDE
:1066A000B11DFFBFBA2FA92F982F88278E0F911DDC
:1066B000A11DB11DE2E0880F991FAA1FBB1FEA951B
:1066C000D1F7861B970B885E9340C8F2215030406B
:1066D0004040504068517C4F21153105410551051E
:1066E00071F60895019739F0880F991F880F991F47
:1066F00002970197F1F70895789484B5826084BD7C
:1067000084B5816084BD85B5826085BD85B58160B5
:1067100085BDEEE6F0E0808181608083E1E8F0E015
:106720001082808182608083808181608083E0E844
:10673000F0E0808181608083E1EBF0E08081846023
:106740008083E0EBF0E0808181608083EAE7F0E025
:106750008081846080838081826080838081816089
:1067600080838081806880831092C1000895CF93D8
:10677000DF93482F50E0CA0186569F4FFC013491A9
:106780004A575F4FFA018491882369F190E0880F9E
:10679000991FFC01E859FF4FA591B491FC01EE58F7
:1067A000FF4FC591D491662351F42FB7F8948C9183
:1067B000932F909589238C93888189230BC0623015
:1067C00061F42FB7F8948C91932F909589238C9333
:1067D0008881832B88832FBF06C09FB7F8948C9144
:1067E000832B8C939FBFDF91CF910895482F50E06A
:1067F000CA0182559F4FFC012491CA0186569F4FC2
:10680000FC0194914A575F4FFA013491332309F404
:1068100040C0222351F1233071F0243028F421307C
:10682000A1F0223011F514C02630B1F02730C1F0AC
:106830002430D9F404C0809180008F7703C0809108
:1068400080008F7D8093800010C084B58F7702C058
:1068500084B58F7D84BD09C08091B0008F7703C05F
:106860008091B0008F7D8093B000E32FF0E0EE0FB9
:10687000FF1FEE58FF4FA591B4912FB7F8946623F0
:1068800021F48C919095892302C08C91892B8C9353
:106890002FBF0895682F70E0CB0182559F4FFC01F8
:1068A0002491CB0186569F4FFC0144916A577F4F3C
:1068B000FB019491992319F420E030E03CC022239D
:1068C00051F1233071F0243028F42130A1F022302E
:1068D00011F514C02630B1F02730C1F02430D9F4BE
:1068E00004C0809180008F7703C0809180008F7DED
:1068F0008093800010C084B58F7702C084B58F7DEF
:1069000084BD09C08091B0008F7703C08091B00032
:106910008F7D8093B000892F90E0880F991F845855
:106920009F4FFC01A591B4918C9120E030E084232D
:1069300011F021E030E0C901089508951F920F92EF
:106940000FB60F9211242F933F934F938F939F93E2
:10695000EF93FF938091C00082FD1DC04091C6005F
:1069600020912E0630912F062F5F3F4F2F733070EE
:1069700080913006909131062817390771F0E09127
:106980002E06F0912F06E251FA4F408330932F06E6
:1069900020932E0602C08091C600FF91EF919F9137
:1069A0008F914F913F912F910F900FBE0F901F909D
:1069B0001895E0918206F0918306E05CFF4F81918B
:1069C000919120813181821B930B8F739070892B61
:1069D00011F00E949D3408951F920F920FB60F92EE
:1069E00011242F933F938F939F93EF93FF932091C5
:1069F000720630917306809174069091750628177F
:106A0000390731F48091C1008F7D8093C10014C09B
:106A1000E0917406F0917506EE5CF94F208180914B
:106A200074069091750601968F7390709093750619
:106A3000809374062093C600FF91EF919F918F91F0
:106A40003F912F910F900FBE0F901F901895DC0172
:106A50001C96ED91FC911D97E05CFF4F21913191C7
:106A600080819181281B390B2F733070C9010895E3
:106A7000DC011C96ED91FC911D97E05CFF4F20819D
:106A80003181E054F040DF01AE5BBF4F8D919C91AE
:106A900011972817390719F42FEF3FEF07C08D9191
:106AA0009C91E80FF91F8081282F30E0C9010895DB
:106AB000DC011C96ED91FC911D97E05CFF4F20815D
:106AC0003181E054F040DF01AE5BBF4F8D919C916E
:106AD00011972817390719F42FEF3FEF10C08D9148
:106AE0009C911197E80FF91F20818D919C9111972E
:106AF00001968F73907011969C938E9330E0C9012C
:106B00000895DC0191968C919197882339F05496E1
:106B1000ED91FC915597808186FFF9CF91961C925B
:106B20000895CF93DF93EC01EE85FF85E05CFF4F86
:106B300020813181E054F0402F5F3F4F2F73307040
:106B4000DF01AE5BBF4F8D919C91119728173907DC
:106B5000D1F3E05CFF4F80819181E054F040E80F79
:106B6000F91F6083EE85FF85E05CFF4F3183208352
:106B7000EE89FF89208181E090E00F8C02C0880FB0
:106B8000991F0A94E2F7282B208381E089A3EC89DE
:106B9000FD8980818064808381E090E0DF91CF91E6
:106BA0000895109279061092780688EE93E0A0E09E
:106BB000B0E080937A0690937B06A0937C06B09316
:106BC0007D0685EF91E090937706809376068EEEB2
:106BD00095E0909383068093820682E396E09093FB
:106BE00085068093840685EC90E0909387068093D9
:106BF000860684EC90E0909389068093880680EC6A
:106C000090E090938B0680938A0681EC90E09093BD
:106C10008D0680938C0682EC90E090938F06809393
:106C20008E0686EC90E0909391068093900684E027
:106C30008093920683E08093930687E08093940686
:106C400085E08093950681E08093960608950F93E2
:106C5000FC0185E092E091838083628343832483F7
:106C600005830F91089585E092E0909399068093B3
:106C7000980610929A0610929B0610929C0610920B
:106C80009D0608958F929F92AF92BF92CF92DF920E
:106C9000EF92FF920F931F93CF93DF934C016B0101
:106CA0007C01AA24BB24C0E0D0E0C601F7016281C8
:106CB0004AE050E00E949D378C01C6016EE20E94BE
:106CC000E636080F191FA00EB11E21960894E11C8C
:106CD000F11CC330D10549F7C601F40165814AE0D2
:106CE00050E00E949D379501280F391FC901DF919F
:106CF000CF911F910F91FF90EF90DF90CF90BF90B9
:106D0000AF909F908F9008959C01FB0185E092E0E9
:106D1000D9018D939C9380819181A281B381F901E6
:106D200082839383A483B5830895FC0185E092E078
:106D30009183808312821382148215820895CF93E7
:106D4000DF930E947C330E94C805C9EDD4E30E9402
:106D500081032097E1F30E94D934F9CFFC0120E0B0
:106D600030E08081882311F421E030E0C9010895EA
:106D7000FC0181E080830895CF92DF92EF92FF9231
:106D80000F931F93CF93DF937C016B018A01C0E0C7
:106D9000D0E00FC0D6016D916D01D701ED91FC914E
:106DA0000190F081E02DC7010995C80FD91F01504E
:106DB00010400115110571F7CE01DF91CF911F91A0
:106DC0000F91FF90EF90DF90CF900895DC01ED914F
:106DD000FC910190F081E02D09950895EF92FF92CA
:106DE0000F931F938C01DC01ED91FC910190F081D8
:106DF000E02D6DE009957C01D801ED91FC910190A9
:106E0000F081E02DC8016AE009959C012E0D3F1D1F
:106E1000C9011F910F91FF90EF900895CF93DF93D9
:106E2000EC016115710519F420E030E00FC0DB01C1
:106E30000D900020E9F71197A61BB70BE881F981A7
:106E40000280F381E02DAD0109959C01C901DF911C
:106E5000CF9108954F925F927F928F929F92AF92BF
:106E6000BF92CF92DF92EF92FF920F931F93DF9327
:106E7000CF93CDB7DEB7A1970FB6F894DEBF0FBEA4
:106E8000CDBF2C01742ECB01223008F42AE019A2C8
:106E900031E2C32ED12CCC0EDD1E822E9924AA24E1
:106EA000BB24672D752FA50194010E94A839790193
:106EB0008A01C801B701A50194010E947539472DC7
:106EC000461B0894C108D1084A3014F4405D01C043
:106ED000495CF6014083E114F1040105110521F03C
:106EE0007E2C5F2DC801DDCFC201B6010E940E3796
:106EF000A1960FB6F894DEBF0FBECDBFCF91DF9144
:106F00001F910F91FF90EF90DF90CF90BF90AF90C7
:106F10009F908F907F905F904F900895DC01211596
:106F2000310541F4ED91FC910190F081E02D642F49
:106F3000099508950E942A370895EF92FF920F93C2
:106F40001F939A01E62EFF2400E010E0B801A7018C
:106F50000E948E371F910F91FF90EF900895CF926E
:106F6000DF92EF92FF920F931F93CF93DF93EC0189
:106F70006A017B012115310541F4E881F981019015
:106F8000F081E02D642F09951FC02A303105D1F41E
:106F900077FF17C0E881F9810190F081E02D6DE263
:106FA00009958C0144275527BA014C195D096E09D2
:106FB0007F09CE012AE00E942A379801280F391F45
:106FC00004C02AE00E942A379C01C901DF91CF91B9
:106FD0001F910F91FF90EF90DF90CF900895EF9267
:106FE000FF920F931F937B019A010027F7FC0095F6
:106FF000102FB801A7010E94AF371F910F91FF908A
:10700000EF9008950E940E370895EF92FF920F932C
:107010001F937C010E940E378C01C7010E94EE363F
:10702000080F191FC8011F910F91FF90EF9008954D
:10703000EF92FF920F931F937B018C0161157105F5
:107040008105910529F420E030E040E050E00BC0DC
:107050000E94E700A80197010E94CA39AC01CB0148
:10706000DA019C01AD01B901CA011F910F91FF9096
:10707000EF900895EF92FF920F931F937B018C0185
:10708000621773078407950764F4261B370B480BB8
:10709000590BCA01B9010E941838E60EF71E081FE5
:1070A000191FB701C8011F910F91FF90EF9008952C
:1070B00098D088F09F5790F0B92F9927B751A0F03A
:1070C000D1F0660F771F881F991F1AF0BA95C9F77C
:1070D00012C0B13081F09FD0B1E008959CC0672FFD
:1070E000782F8827B85F39F0B93FCCF3869577952C
:1070F0006795B395D9F73EF4909580957095619515
:107100007F4F8F4F9F4F0895E89409C097FB3EF43F
:1071100090958095709561957F4F8F4F9F4F9923E4
:10712000A9F0F92F96E9BB279395F6958795779562
:107130006795B795F111F8CFFAF4BB0F11F460FF22
:107140001BC06F5F7F4F8F4F9F4F16C0882311F07A
:1071500096E911C0772321F09EE8872F762F05C08E
:10716000662371F096E8862F70E060E02AF09A9529
:10717000660F771F881FDAF7880F9695879597F91E
:10718000089597F99F6780E870E060E008959FEFA9
:1071900080EC089500240A941616170618060906AE
:1071A000089500240A94121613061406050608957D
:1071B000092E0394000C11F4882352F0BB0F40F405
:1071C000BF2B11F460FF04C06F5F7F4F8F4F9F4F45
:1071D000089557FD9058440F551F59F05F3F71F0C7
:1071E0004795880F97FB991F61F09F3F79F087952E
:1071F0000895121613061406551FF2CF4695F1DFB7
:1072000008C0161617061806991FF1CF8695710546
:10721000610508940895E894BB2766277727CB017A
:1072200097F908950BD0C4CFB5DF28F0BADF18F076
:10723000952309F0A6CFABCF1124EECFCADFA0F380
:10724000959FD1F3950F50E0551F629FF001729FFB
:10725000BB27F00DB11D639FAA27F00DB11DAA1F1A
:10726000649F6627B00DA11D661F829F2227B00D67
:10727000A11D621F739FB00DA11D621F839FA00DF2
:10728000611D221F749F3327A00D611D231F849F42
:10729000600D211D822F762F6A2F11249F57504099
:1072A0008AF0E1F088234AF0EE0FFF1FBB1F661F34
:1072B000771F881F91505040A9F79E3F510570F0ED
:1072C00060CFAACF5F3FECF3983EDCF386957795CD
:1072D0006795B795F795E7959F5FC1F7FE2B880FE8
:1072E000911D9695879597F90895629FD001739F98
:1072F000F001829FE00DF11D649FE00DF11D929F52
:10730000F00D839FF00D749FF00D659FF00D992790
:10731000729FB00DE11DF91F639FB00DE11DF91FB4
:10732000BD01CF0111240895AA1BBB1B51E107C069
:10733000AA1FBB1FA617B70710F0A61BB70B881F05
:10734000991F5A95A9F780959095BC01CD01089594
:10735000A1E21A2EAA1BBB1BFD010DC0AA1FBB1F59
:10736000EE1FFF1FA217B307E407F50720F0A21BCB
:10737000B30BE40BF50B661F771F881F991F1A9438
:1073800069F760957095809590959B01AC01BD0162
:10739000CF01089597FB092E05260ED057FD04D086
:1073A000D7DF0AD0001C38F45095409530952195D0
:1073B0003F4F4F4F5F4F0895F6F79095809570952A
:1073C00061957F4F8F4F9F4F0895EE0FFF1F0590E0
:1073D000F491E02D09942F923F924F925F926F9219
:1073E0007F928F929F92AF92BF92CF92DF92EF9255
:1073F000FF920F931F93CF93DF93CDB7DEB7CA1BD6
:10740000DB0B0FB6F894DEBF0FBECDBF09942A8800
:10741000398848885F846E847D848C849B84AA84A8
:10742000B984C884DF80EE80FD800C811B81AA8135
:10743000B981CE0FD11D0FB6F894DEBF0FBECDBF00
:10744000ED010895F894FFCF474554202F617264F1
:1074500075696E6F2F6176725F72662E7068703F0D
:107460006164723D0026766F6C3D00204854545094
:107470002F312E3100486F73743A206133332E77E9
:107480002E707700557365722D4167656E743A20D2
:1074900061726475696E6F2D65746865726E65746E
:1074A00000436F6E6E656374696F6E3A20636C6F34
:1074B000736500454E4332384A0001000000DEADDE
:1074C000BEEFFEED6133332E772E7077006F75744B
:1074D0000030303030303030303030000101400189
:1074E000FF3C000000000014140E148A11E210A9E1
:1074F000121D118D142814D8128213B5106B13CCE1
:10750000109910000000001A188D1906193218324F
:10751000191219711A9F1AD719D71AA819201958B0
:10752000191218EC187B1800000000FFFFFFFFFF86
:10753000FFFFFFFFFFFFFFFFFF000000009135BCD2
:107540003627355835383581350000000042360081
:107550000030303030303030303030000101400108
:10756000FF3C000000000014140E148A11E210A960
:10757000121D118D142814D8128213B5106B13CC60
:10758000FFFFFFFFFFFFFFFFFFFFFFFFFFFFFFFF0B
:10759000FFFFFFFFFFFFFFFFFFFFFFFFFFFFFFFFFB
:1075A000FFFFFFFFFFFFFFFFFFFFFFFFFFFFFFFFEB
:1075B000FFFFFFFFFFFFFFFFFFFFFFFFFFFFFFFFDB
:107E0000112484B714BE81FFF0D085E080938100F7
:107E100082E08093C00088E18093C10086E0809377
:107E2000C20080E18093C4008EE0C9D0259A86E02C
:107E300020E33CEF91E0309385002093840096BBD3
:107E4000B09BFECF1D9AA8958150A9F7CC24DD24C4
:107E500088248394B5E0AB2EA1E19A2EF3E0BF2EE7
:107E6000A2D0813461F49FD0082FAFD0023811F036
:107E7000013811F484E001C083E08DD089C08234E0
:107E800011F484E103C0853419F485E0A6D080C0E4
:107E9000853579F488D0E82EFF2485D0082F10E0AE
:107EA000102F00270E291F29000F111F8ED06801E7
:107EB0006FC0863521F484E090D080E0DECF843638
:107EC00009F040C070D06FD0082F6DD080E0C81688
:107ED00080E7D80618F4F601B7BEE895C0E0D1E017
:107EE00062D089930C17E1F7F0E0CF16F0E7DF06D8
:107EF00018F0F601B7BEE89568D007B600FCFDCFD4
:107F0000A601A0E0B1E02C9130E011968C91119780
:107F100090E0982F8827822B932B1296FA010C0160
:107F200087BEE89511244E5F5F4FF1E0A038BF0790
:107F300051F7F601A7BEE89507B600FCFDCF97BE46
:107F4000E89526C08437B1F42ED02DD0F82E2BD052
:107F50003CD0F601EF2C8F010F5F1F4F84911BD097
:107F6000EA94F801C1F70894C11CD11CFA94CF0C13
:107F7000D11C0EC0853739F428D08EE10CD085E9AC
:107F80000AD08FE07ACF813511F488E018D01DD067
:107F900080E101D065CF982F8091C00085FFFCCF94
:107FA0009093C60008958091C00087FFFCCF809118
:107FB000C00084FD01C0A8958091C6000895E0E648
:107FC000F0E098E1908380830895EDDF803219F02E
:107FD00088E0F5DFFFCF84E1DECF1F93182FE3DFCA
:107FE0001150E9F7F2DF1F91089580E0E8DFEE27F6
:107FF000FF270994FFFFFFFFFFFFFFFFFFFF0404C0
:00000001FF
